:10000000FCC4000028C5000026C5000024C500006F
:100010000C948C1120C500000C94180E0C94640DE7
:100020001AC5000018C5000016C5000014C5000060
:1000300012C5000010C500000EC500000CC5000070
:100040000AC5000008C500000C942D2E04C5000050
:1000500002C5000000C50000FEC40000FCC4000092
:10006000FAC40000F8C40000F6C40000F4C40000A4
:10007000F2C40000F0C40000EEC40000ECC40000B4
:10008000EAC40000E8C40000E6C40000787C3C1E1E
:100090001E1E1E1E3E3EFEFCFCF8F0E0800000002E
:1000A00000000000000080E0FFFFFFFF7F1F000056
:1000B0000000FFFFFFFFFF0707030301010000002F
:1000C00000000078FCFCFCFC780000000000000050
:1000D000000000C020100808040202020101010112
:1000E000F00E0100000000000060707000000000D1
:1000F0000F708000000000008040201010080808E9
:1001000000000003040810102040404080808080E0
:100110000F708000000000000810204040808080A8
:1001200020205072657373205245534554206275E8
:1001300074746F6E00202044656661756C74204D88
:100140006F646520536176656400204861726420A5
:100150004469736B202020202020202020202000B4
:1001600020466C6F7070792044726976652020207B
:10017000202020202000504C454153452057414924
:1001800054003130313031303130313031302E2E79
:100190002E0030313031303130313031303130318A
:1001A0003000202020205550444154494E472043E0
:1001B000504C442020202000436F6E747261737491
:1001C0003A200053454C4543543A2053617665002C
:1001D0004E4558543A204461726B65720050524546
:1001E000563A204C69676874657200626567696E8B
:1001F0000052656C6561736520627574746F6E730F
:1002000020746F00434F4E54524153542041444A8E
:100210005553544D454E54004170702056657273CD
:10022000696F6E20302E3720420053454C454354B1
:100230003A20436F6E666967204D656E7500466CA7
:100240006F707079204472697665204D6F64650027
:1002500048617264204469736B204D6F64650020AF
:1002600020202020464C4F50505920454D552020ED
:100270002020202000534420524541442045525222
:100280004F522052006669726D776172652E7876E2
:100290006600202020202020202020202020202038
:1002A00020202020202000436F756C64206E6F7426
:1002B000206F70656E00464154414C204552524FAC
:1002C0005220202020202020202020005752495456
:1002D00045204552524F522020202020202020200F
:1002E000200000000C001800240030003C004800F2
:1002F000540060006C007800840090009C00A8000E
:10030000B400C000CB00D600E100EC00F700020111
:100310000D01180123012E01390144014F015A0139
:10032000650170017A0184018E019801A201AC017E
:10033000B601C001CA01D401DE01E801F201FC01ED
:1003400006021002190222022B0234023D0246026A
:100350004F02580261026A0273027C0285028E0219
:100360009702A002A802B002B802C002C802D002DE
:10037000D802E002E802F002F802000308031003CA
:1003800018030C0C0C0C0C0C0C0C0C0C0C0C0C0CAA
:100390000C0C0B0B0B0B0B0B0B0B0B0B0B0B0B0BAB
:1003A0000B0B0A0A0A0A0A0A0A0A0A0A0A0A0A0AAB
:1003B0000A0A0909090909090909090909090909AB
:1003C00009090808080808080808080808080808AB
:1003D000080896979A9B9D9E9FA6A7ABACADAEAF23
:1003E000B2B3B4B5B6B7B9BABBBCBDBEBFCBCDCE48
:1003F000CFD3D6D7D9DADBDCDDDEDFE5E6E7E9EA25
:10040000EBECEDEEEFF2F3F4F5F6F7F9FAFBFCFDA9
:10041000FEFF0001FFFF0203FF040506FFFFFFFFD1
:10042000FFFF0708FFFFFF090A0B0C0DFFFF0E0F70
:1004300010111213FF1415161718191AFFFFFFFFDA
:10044000FFFFFFFFFFFFFF1BFF1C1D1EFFFFFF1F26
:10045000FFFF2021FF22232425262728FFFFFFFF5F
:10046000FF292A2BFF2C2D2E2F303132FFFF333462
:1004700035363738FF393A3B3C3D3E3F00002110CE
:10048000422063308440A550C660E77008812991FE
:100490004AA16BB18CC1ADD1CEE1EFF131121002A6
:1004A00073325222B5529442F772D662399318834E
:1004B0007BB35AA3BDD39CC3FFF3DEE36224433472
:1004C00020040114E664C774A44485546AA54BB59E
:1004D00028850995EEE5CFF5ACC58DD55336722646
:1004E00011163006D776F6669556B4465BB77AA7EE
:1004F00019973887DFF7FEE79DD7BCC7C448E55892
:100500008668A7784008611802282338CCC9EDD93D
:100510008EE9AFF9488969990AA92BB9F55AD44AE5
:10052000B77A966A711A500A333A122AFDDBDCCB8D
:10053000BFFB9EEB799B588B3BBB1AABA66C877CB1
:10054000E44CC55C222C033C600C411CAEED8FFDDD
:10055000ECCDCDDD2AAD0BBD688D499D977EB66E85
:10056000D55EF44E133E322E511E700E9FFFBEEF2D
:10057000DDDFFCCF1BBF3AAF599F788F8891A981EF
:10058000CAB1EBA10CD12DC14EF16FE18010A100D9
:10059000C230E3200450254046706760B9839893C9
:1005A000FBA3DAB33DC31CD37FE35EF3B102901229
:1005B000F322D2323542145277625672EAB5CBA595
:1005C000A89589856EF54FE52CD50DC5E234C32479
:1005D000A01481046674476424540544DBA7FAB769
:1005E0009987B8975FE77EF71DC73CD7D326F236C9
:1005F0009106B01657667676154634564CD96DC9B5
:100600000EF92FE9C899E9898AB9ABA94458654818
:1006100006782768C018E1088238A3287DCB5CDB08
:100620003FEB1EFBF98BD89BBBAB9ABB754A545A68
:10063000376A167AF10AD01AB32A923A2EFD0FEDD4
:100640006CDD4DCDAABD8BADE89DC98D267C076CB8
:10065000645C454CA23C832CE01CC10C1FEF3EFFA8
:100660005DCF7CDF9BAFBABFD98FF89F176E367E08
:10067000554E745E932EB23ED10EF01E20202020E7
:10068000202020202020202020202020202020206A
:1006900020002049646C6500205265616400577237
:1006A00069746500547261636B2020202053696473
:1006B0006500313434304B204469736B436F70797B
:1006C00020696D616765003830304B204469736B79
:1006D000436F707920696D616765003430304B205D
:1006E0004469736B436F707920696D616765003190
:1006F0003434304B2072617720696D616765003852
:1007000030304B2072617720696D6167650034304D
:10071000304B2072617720696D6167650066696C96
:1007200065206E6F7420636F6E746967756F757383
:10073000006572726F72206F70656E696E672069F6
:100740006D61676500434845434B2050494E532037
:100750002D2044454641554C5400434845434B20C9
:1007600050494E20434C4B4F2D4800434845434B86
:100770002050494E20434C4B4F2D4C00434845439D
:100780004B2050494E205245534554000000000074
:100790000000000000000000000000000000000059
:1007A0000000000000000000000000000000000049
:1007B0000000000000000000000000000000000039
:1007C0000000000000000000000000000000000029
:1007D000000000007FFFFFFE80000001800000019C
:1007E0008000000180000001800000018000000105
:1007F0008800000180000001800000017FFFFFFEF3
:1008000000000000000000000000000000000000E8
:1008100000000000000000000000000000000000D8
:1008200000000000000000000000000000000000C8
:1008300000000000000000000000000000000000B8
:1008400000000000000000000000000000000000A8
:10085000000000007FFFFFFEFFFFFFFFFFFFFFFF25
:10086000FFFFFFFFFFFFFFFFFFFFFFFFFFFFFFFF98
:10087000FFFFFFFFFFFFFFFFFFFFFFFF7FFFFFFE09
:10088000000000000000000000000000484432307A
:10089000204469736B20456D756C6174696F6E00DF
:1008A00066696C65206E6F7420636F6E746967751E
:1008B0006F757300466C6F70707920456D750044DC
:1008C000495341424C45440000000000170003001A
:1008D000031F0A1F0A1F050904120F171C00030338
:1008E000000E11110E00050205040E04100800048C
:1008F00004040010001804031E110F021F00191534
:100900001215150A07041F1715091E151D190503D1
:100910001A150B17150F000A00040C04040E1F0A09
:100920000A0A1F0E040115030E15161E051E1F15BB
:100930000A0E11111F110E1F15151F05050E151D8D
:100940001F041F111F1108100F1F041B1F10101F61
:10095000061F1F0E1F0E110E1F05020E191E1F0D62
:1009600016121509011F010F101F0718071F0C1F72
:100970001B041B031C031915131F1010020408107D
:10098000101F0406041010100003031A161C1F1277
:100990000C0C12120C121F0C1A16041E050C2A1E27
:1009A0001F021C001D0010201D1F0C12111F101E05
:1009B0000E1E1E021C0C120C3E120C0C123E1C02CF
:1009C00002141E0A021F120E101E0E180E1E1C1EEE
:1009D000120C1206281E1A1F16041B11001F0011EC
:1009E0001B04080C047C3C3E5E2B3D3F2F5B5D3BB3
:1009F0002C2A225C00002B0C2E0C11241FBECFEFE2
:100A0000D0E4DEBFCDBF15E0A0E0B1E0ECEBFBE948
:100A100000E00BBF02C007900D92A431B107D9F7D7
:100A200019E3A4E1B5E001C01D92A83FB107E1F7C9
:100A300019E000E0C8EFD9E040E006C02297410984
:100A4000FE014BBF0E94754AC63FD1074007B1F770
:100A5000C6D50C94CD4DD4CA8130910559F000977C
:100A600021F480914405882309F4089581E495E0F8
:100A70000C940F3810924105109244050895FF928E
:100A80000F931F93CF93DF938C01F0902D05C091AE
:100A90002E05D0912F0580914005882309F459C077
:100AA0000E94CC260E94C02F80E060E00E946D2E44
:100AB000FF2009F43FC08CEC92E061E00E94152F0A
:100AC00080E061E00E946D2EC80160E044E50E9474
:100AD000942E8DB79EB708970FB6F8949EBF0FBEA1
:100AE0008DBFEDB7FEB7319606E115E0ADB7BEB7E5
:100AF00012961C930E93119786E190E09383828364
:100B000080E091E095838483D783C6830E94D34A93
:100B10008DB79EB708960FB6F8949EBF0FBE8DBFD7
:100B200080E065E00E946D2EC80160E044E50E940F
:100B3000942EFFCF86EB92E061E00E94152F80E0BB
:100B400061E00E946D2EC80160E044E50E94942E91
:100B5000F0CF0E94B815A6CF20915C3530915D355D
:100B600082E02030380771F0E0915E35F0915F351A
:100B7000E20FF31F80812F5F3F4F30935D3520934D
:100B80005C35089560915E3570915F3581E495E044
:100B900040E052E00E94A53597FD0BC010925D35F4
:100BA00010925C3585B198E0892785B920E030E066
:100BB000DBCF83E091E063DFF1CFDF92EF92FF9232
:100BC0000F931F93CF93DF93082F2B9880914005AD
:100BD000882309F47EC00E94BA1D0E94CC2FC6E172
:100BE000D5E0FE0101900020E9F73197EC1BFD0BE9
:100BF0008E2F8195880F865D65E00E946D2ECE0157
:100C000060E044E50E94942E0E94262E002309F401
:100C100038C000ED10E0DD2480E06D2D0E946D2EC7
:100C20002AE1E22E81E060E00E945E2EEA94D1F794
:100C300090E1E92EF12CE00EF11EE801FE01649135
:100C400081E00E945E2E2196EC16FD06B9F7E801C0
:100C50002F9601501040FE01649181E00E945E2EAB
:100C600021970C171D07B9F70AE181E060E00E94A7
:100C70005E2E0150D1F7D394FD2DF43061F1870140
:100C8000CBCFCCE8D0E0FF2480E06F2D0E946D2E0A
:100C900001E281E060E00E945E2E0150D1F78E01FA
:100CA0000F5E1F4FFE01649181E00E945E2E21962F
:100CB0000C171D07B9F782E2E82E81E060E00E9480
:100CC0005E2EEA94D1F7F394FF2DF43021F0E80181
:100CD000DBCFC7D582CF98E02FEB37E249E0215038
:100CE00030404040E1F700C0000085B1892785B958
:100CF000F3CFBF92CF92DF92EF92FF920F931F93A9
:100D0000CF93DF9387E893E10197F1F700C00000EC
:100D100029E0E0E0F0E0209357006491A7E8B3E118
:100D20001197F1F700C00000E3E0F0E020935700D6
:100D3000849190E0E7E8F3E13197F1F700C000001B
:100D4000E2E0F0E020935700249130E0A7E8B3E11F
:100D50001197F1F700C000008A3D910509F4FAC02F
:100D6000823D910509F4F6C0EDB7FEB73C970FB68A
:100D7000F894FEBF0FBEEDBF319656E1E52E55E06B
:100D8000F52EADB7BEB71296FC92EE92119746E1E2
:100D900050E05383428343E151E0558344836683AB
:100DA000178291878087338722870E94D34AEDB7C5
:100DB000FEB73C960FB6F894FEBF0FBEEDBF81E0C4
:100DC000FCDE20912C052F3709F4D4C02E3041F1E0
:100DD0004DB75EB7485050400FB6F8945EBF0FBE97
:100DE0004DBFEDB7FEB73196ADB7BEB71296FC92C8
:100DF000EE92119786E190E0938382838AE391E0FB
:100E000095838483268317820E94D34AEDB7FEB769
:100E100038960FB6F894FEBF0FBEEDBF81E0CDDE71
:100E200080914005882309F4C8C000ED10E0DD245E
:100E300080E06D2D0E946D2E4AE1C42E81E060E0BD
:100E40000E945E2ECA94D1F7C02EB12EC0E0D0E031
:100E50000CC0EC2DFB2DEC0FFD1F649181E00E9476
:100E60005E2E2196C031D10531F0FD2DF23089F78B
:100E7000E0E1F1E0F0CFCFE0D0E00DC0EC2DFB2DB4
:100E8000EC0FFD1F649181E00E945E2E21975FEFC1
:100E9000CF3FD50731F04D2D423081F7E0E1F1E051
:100EA000EFCF3AE1C32E81E060E00E945E2ECA944B
:100EB000D1F7D394005F1F4F8D2D843009F0B8CF48
:100EC00000D000D000D0EDB7FEB73196ADB7BEB7B9
:100ED0001296FC92EE92119786E190E093838283C2
:100EE0008AE491E0958384830E94D34AF7010190BC
:100EF0000020E9F73197E651F5404DB75EB74A5FFC
:100F00005F4F0FB6F8945EBF0FBE4DBF8E2F819519
:100F1000880F865D65E00E946D2EC70160E044E5A4
:100F20000E94942E2B988FEF93EDA0E38150904078
:100F3000A040E1F700C0000085B198E0892785B99D
:100F4000DF91CF911F910F91FF90EF90DF90CF90A5
:100F5000BF9008952C3F310521F02F3F310509F056
:100F600003CF66E1E62E65E0F62E20912C052F37A3
:100F700009F02CCF00D000D000D0EDB7FEB73196ED
:100F8000ADB7BEB71296FC92EE92119786E190E053
:100F9000938382838CE291E0958384830E94D34A79
:100FA000EDB7FEB736960FB6F894FEBF0FBEEDBF95
:100FB00080E003DE20912C0509CF96D436CF1F9315
:100FC000CF93DF938FEF99E6A8E181509040A04046
:100FD000E1F700C0000081E495E067E571E041E0E1
:100FE0000E94103B882309F470C06CE575E0709393
:100FF0005F3560935E3581E495E040E052E00E9409
:10100000A53597FD7FC010925D3510925C358CEA56
:1010100095E00E94A5491FB7F8940E944F49EC0142
:101020001FBF81E495E00E940F380E94C02F2097D7
:1010300059F1ADB7BEB718970FB6F894BEBF0FBE43
:10104000ADBFEDB7FEB7319686E195E012969C9361
:101050008E93119786E190E09383828384E791E0F9
:1010600095838483D783C6830E94D34A8DB79EB766
:1010700008960FB6F8949EBF0FBE8DBF81E09DDD30
:10108000DF91CF911F91089589E062E00E946D2E5B
:1010900086E195E064E671E046E150E00E94C44AD2
:1010A00086E195E060E044E50E94942E8FEF9AE19E
:1010B000A7EB81509040A040E1F700C00000FE0186
:1010C0000995DF91CF911F91089564E00E946D2EE4
:1010D00087EA92E060E00E94152F80E065E00E94C0
:1010E0006D2E82E992E060E00E94152F86E195E086
:1010F00065E872E00E94814A80E05FDDDF91CF9178
:101100001F91089586E195E065E772E00E94814AAB
:1011100081E053DD78CFCF93DF930E94C02F80E032
:1011200060E00E946D2E8FE592E061E00E94152F35
:1011300088E192E00E94884A8195880F865D62E08E
:101140000E946D2E88E192E060E00E94152F4DB75D
:101150005EB7485050400FB6F8945EBF0FBE4DBF0B
:10116000EDB7FEB73196C6E1D5E0ADB7BEB7129682
:10117000DC93CE93119786E190E09383828386E897
:1011800091E09583848380912C05868317820E9449
:10119000D34AFE0101900020E9F73197EC1BFD0BCB
:1011A0004DB75EB7485F5F4F0FB6F8945EBF0FBE96
:1011B0004DBF8E2F8195880F865D63E00E946D2E56
:1011C000CE0160E044E50E94942E80914005882382
:1011D00009F44AC0C0E5D2E0CE010E94884A819558
:1011E000880F865D61E00E946D2ECE0160E00E9456
:1011F000152F8AE292E00E94884A8195880F865DC9
:1012000065E00E946D2E8AE292E060E00E94152F58
:101210000E94262E94E028E08AE04FEF51EE64E031
:10122000415050406040E1F700C00000499B0FC0B2
:101230004A9B0DC04C990BC04FE75FE462E14150FF
:1012400050406040E1F700C000004A9910C0815052
:1012500021F785B1822785B99150F1F60E942A2E97
:1012600080E0DF91CF910895CEE3D2E0B5CF0E9428
:101270002A2E2B9881E0DF91CF910895CF92DF92B3
:10128000EF92FF920F931F93DF93CF9300D000D084
:10129000CDB7DEB780E060E00E946D2E0E94C02FC7
:1012A00080E060E00E946D2E84E092E060E00E94A9
:1012B000152F80E062E00E946D2E81EF91E060E0EA
:1012C0000E94152F80E063E00E946D2E8BEE91E06E
:1012D00060E00E94152F499BFECF4A9BFCCF4C9BA0
:1012E000FACF80E060E00E946D2E0E94C02F80E067
:1012F00062E00E946D2E8DED91E060E00E94152F5E
:1013000080E063E00E946D2E80ED91E060E00E943D
:10131000152F80E064E00E946D2E83EC91E060E088
:101320000E94152F8E010F5F1F4FE7E9EE2EE1E0BF
:10133000FE2E74E0C72ED12C16C08091E2378F3F6D
:1013400029F08091E2378F5F8093E23780E061E29D
:101350000E945E2E6091E23780E00E945E2E80E067
:1013600060E20E945E2E80E060E00E946D2E88EBBD
:1013700091E060E00E94152F8091E2372DB73EB7D3
:10138000285030400FB6F8943EBF0FBE2DBFEDB7CA
:10139000FEB73196ADB7BEB712961C930E93119758
:1013A000D382C282F582E482868317820E94D34A66
:1013B0002DB73EB7285F3F4F0FB6F8943EBF0FBE24
:1013C0002DBFC80160E044E50E94942E8FEF99E69E
:1013D000A8E181509040A040E1F700C00000499B87
:1013E00004C04A9B02C04C99FACF4A9BA6CF4999A8
:1013F0000BC08091E237813808F4A8CF8091E237A2
:1014000081508093E237A2CF4C99A0CF6091E23710
:1014100081E090E00E941B4D8FEF99E6A8E181509A
:101420009040A040E1F700C000000E94C02F0F9044
:101430000F900F900F90CF91DF911F910F91FF9020
:10144000EF90DF90CF90089580E060E00E946D2ED5
:101450000E94C02F80E060E00E946D2E82EA91E041
:1014600061E00E94152F89E062E00E946D2E82E902
:1014700091E060E00E94152F89E063E00E946D2EEC
:1014800082E891E060E00E94152F8FE065E00E9405
:101490006D2E86E791E060E00E94152F90CDCF93EE
:1014A000DF9380E060E00E946D2E81E06FE70E9494
:1014B0005E2EC4E0D0E081E060E40E945E2E2197C1
:1014C000D1F78AE991E00E947D2F81E060E40E94DB
:1014D0005E2E81E060E40E945E2E81E06FE70E9454
:1014E0005E2E80E062E00E946D2E6091400581E0FA
:1014F000682780E691E00E94152F80E063E00E945B
:101500006D2E8AE491E0609140050E94152FDF91D5
:10151000CF9108950F931F938FE79AE1A6E0815032
:101520009040A040E1F700C000004C9BFECF8FE749
:101530009AE1A6E081509040A040E1F700C0000091
:10154000AEDF1091400501E0499B2CC04A9B37C09B
:101550004C99FACF0E94C02F8FEF94E3ACE08150FA
:101560009040A040E1F700C000004C9BFECF60918E
:101570004005161789F182E090E00E941B4D80E043
:1015800061E00E946D2E85E391E060E00E94152FDE
:1015900080E063E00E946D2E80E291E060E00E94B6
:1015A000152FFFCF109240057ADF8FEF94E3ACE068
:1015B00081509040A040E1F700C00000C5CF0093EB
:1015C00040056DDF8FEF94E3ACE081509040A04088
:1015D000E1F700C00000B8CF1F910F910895BF92AE
:1015E000CF92DF92EF92FF920F931F93DF93CF93EF
:1015F000CDB7DEB7ED970FB6F894DEBF0FBECDBF07
:10160000E0911505F0E0EE0FFF1FE850F0418081FA
:101610008093140580E090E00E94134D10924005E5
:10162000823F09F4FAC0813F09F401C180E090E0F3
:1016300062EF0E941B4D81E090E064EB0E941B4D25
:1016400082E090E0609140050E941B4D0E94202E98
:1016500080914005882309F468C00E94CC26499BEC
:1016600002C04A9B71C0499B63C043DB8091400527
:10167000882309F466C078948FE79AE1A6E0815048
:101680009040A040E1F700C000000E94262E8FE7A6
:101690009AE1A6E081509040A040E1F700C0000030
:1016A00089E189831C821C8E1BA21EA28E010F5F02
:1016B0001F4FC80161E00E94923BE82E2CDDB82E3E
:1016C0000E94C02F499B04C04A9902C04C9BC1C0D4
:1016D000EE2009F444C00E942A2E499904C04A9978
:1016E00002C04C99B4C0BB20C1F58091400588234D
:1016F00081F1C8010E940C278EA1882321F0CE0120
:1017000083960E940F3880E090E0ED960FB6F89433
:10171000DEBF0FBECDBFCF91DF911F910F91FF9024
:10172000EF90DF90CF90BF9008950E94B81597CFAB
:101730004A999BCF4C9B99CF80914005882309F013
:101740009ACF0E94051697CF4C9B90CF49998DCF89
:10175000EFCFC8010E94F718CFCFDCDEC6CF00D094
:1017600000D000D0EDB7FEB73196B6E1EB2EB5E074
:10177000FB2EADB7BEB71296FC92EE921197A6E182
:10178000CA2ED12CD382C2828EEA91E095838483C3
:101790000E94D34AF70101900020E9F73197EE1932
:1017A000FF098DB79EB706960FB6F8949EBF0FBE81
:1017B0008DBF8E2F8195880F865D64E00E946D2E0F
:1017C000C70160E044E50E94942EADB7BEB71A97FA
:1017D0000FB6F894BEBF0FBEADBFEDB7FEB73196E2
:1017E0001296FC92EE921197D382C2828AEB91E01C
:1017F000958384838981868317828B818087118674
:101800000E94D34A8DB79EB70A960FB6F8949EBF32
:101810000FBE8DBF80E0D1D95ECF82E090E00E9404
:10182000134D91E0882379F0909340050FCF80E02D
:1018300090E062EF0E941B4D82E090E060914005D5
:101840000E941B4D03CF90E090934005FFCEFCDD3E
:101850004ACF14DD3DCF81E090E0FEC880E090E00B
:10186000FBC882E282B95D98429A289A4598089509
:101870000F9336B191E0811190E0331F3327331F6E
:10188000931759F0E9B1E095E170F0E081E090E064
:10189000662331F4E817F90741F080E00F910895CD
:1018A00080E090E0E817F907C1F766B160956170D4
:1018B00070E081E090E0442311F080E090E0681750
:1018C000790759F790B181E0211180E0991F99279C
:1018D000991F891711F329B191E0011190E081E07E
:1018E00023FF80E08927DACF0F93CF93DF934899C6
:1018F00086C0459A11B8469A8FEF9FEF03C00197B3
:1019000009F489C0079BFBCF8FEF9FEF03C00197BE
:1019100009F48AC00799FBCF459846988FE781B9AB
:1019200081E060E041E020E000E0A2DF882321F0D8
:10193000DF91CF910F91089546B129B186B1B0B131
:10194000A9B16DB77EB7605170400FB6F8947EBFF5
:101950000FBE6DBFEDB7FEB7319666E175E0CDB74E
:10196000DEB77A83698366E170E0738362836BEC30
:1019700071E075836483552747FD5095952F991F16
:101980009927991F9683178230E021703070208745
:10199000118690E081709070828713868B2F992733
:1019A00087FD9095892F881F8827881F8487158633
:1019B00081E090E0A3FF2CC0978786870E94D34ADE
:1019C0006DB77EB7605F7F4F0FB6F8947EBF0FBED6
:1019D0006DBF80E064E00E946D2E86E195E060E0DE
:1019E00044E50E94942E86E195E065E477E00E944C
:1019F000814A81E0E2D8DF91CF910F91089586E18D
:101A000095E06CE777E00E94814A81E0D6D871CFFB
:101A100080E090E0D1CF86E195E06BE677E00E9430
:101A2000814A81E0CAD870CF86E195E06AE577E027
:101A30000E94814A81E0C1D86FCF1F93DF93CF937B
:101A4000CDB7DEB72A970FB6F894DEBF0FBECDBF75
:101A5000CE010196DC01E1E3F3E02AE001900D9272
:101A60002150E1F7E0916035F0E0F595E795F595C7
:101A7000E795F595E795F595E7951FB7F894E53067
:101A800008F0E4E0F0E0EE0FFF1FE80FF91F2081FF
:101A90003181220F331F40E050E060E07DE281E3BE
:101AA00091E00E945A4A30936C3520936B351FBFEA
:101AB00082E086BB2A960FB6F894DEBF0FBECDBF7C
:101AC000CF91DF911F9108951F920F920FB60F9241
:101AD0000BB60F9211242F933F934F935F936F9305
:101AE0007F938F939F93AF93BF93CF93DF93EF93A6
:101AF000FF93489B2FC0E091603580916635882325
:101B000009F03DC0F0E0EE57FC4F249130E0220F89
:101B1000331F21153105A9F537995DC080916035D6
:101B20008F5F8093603580916035882309F064C0B1
:101B30004598429A4899FECF4298459A7EDFC091D7
:101B40003205D0913305C330D10508F057C081E08C
:101B500080936435FF91EF91DF91CF91BF91AF9169
:101B60009F918F917F916F915F914F913F912F91B5
:101B70000F900BBE0F900FBE0F901F90189524E290
:101B800030E080E090E040E050E068E18159984C1E
:101B9000FC01808180FF03C0683159F1542F4F5FF1
:101BA000842F90E0821793070CF1561708F4B4CFF6
:101BB000862FE82FF0E0E159F84C908191FF03C0A7
:101BC0009081916090839081946090838F5F58178B
:101BD00080F7379BA3CF80916035882309F4A3CF8A
:101BE000809160358150809360359DCF4831E9F216
:101BF000CDCF542F642FD3CF459A9BCF86E195E06C
:101C00006DED71E046E150E00E94C44AC851DC4FDE
:101C1000D0932F05C0932E051092300581E080935C
:101C2000643580932D0510923305109232058FCFC5
:101C30001F920F920FB60F920BB60F9211241F93A3
:101C40002F933F934F935F936F937F938F939F93C4
:101C5000AF93BF93CF93DF93EF93FF9386B190E061
:101C600095958795817090916235891791F0909143
:101C70006935923009F46DC01092623511E010930D
:101C80006435C0913205D0913305C330D10508F0D9
:101C900047C086B1817011E0812790913005891786
:101CA000C9F08093300580913005882349F5469826
:101CB0008FE781B980916B008F7780936B00C09123
:101CC0003205D0913305C330D10508F045C081E01D
:101CD00080936435FF91EF91DF91CF91BF91AF91E8
:101CE0009F918F917F916F915F914F913F912F9134
:101CF0001F910F900BBE0F900FBE0F901F90189565
:101D000011B8469A80916B00806880936B0080B117
:101D10008078809331051092330510923205D7CF29
:101D200086E195E06DED71E046E150E00E94C44A25
:101D3000C053D84FD0932F05C0932E051092300575
:101D40001093643510932D051092330510923205CF
:101D5000A0CF8093623592CF86E195E06DED71E082
:101D600046E150E00E94C44AC854D44FD0932F0596
:101D7000C0932E05109230051093643510932D05F5
:101D80001092330510923205A2CF1F93E0B1E068A4
:101D900080913205909133058430910588F4833029
:101DA000910509F487C0DC01AE5DBC4F2C912E1764
:101DB00009F404C110923305109232051F91089561
:101DC000F0E0E458FC4FE49132E08F3B930748F594
:101DD0009C01237030702230310509F4BBC02330E0
:101DE000310509F449C12130310509F418C1EE0F5C
:101DF000EE0FE0938A3740918E3750E09A01220F20
:101E0000232F221F330B20938F37440F551F422B54
:101E100040938E37019690933305809332051F913E
:101E20000895F2E08F3B9F0709F4C1C022E0803C97
:101E3000920709F4CEC032E0813C930709F4E2C175
:101E4000F2E0823C9F0709F0B5CF80918A37982F46
:101E5000990F990F90938A37E82B90918E37E91755
:101E6000C9F086E195E06EE372E046E150E00E9441
:101E7000C44A80E490E090932F0580932E05109241
:101E8000300581E08093643580932D0510923305F1
:101E900010923205E0918B37F0E0E159F84C8081E7
:101EA0008260808380818160808380818B7F80835A
:101EB0002B9A80CFF0E0E458FC4F1491E09160350C
:101EC00080916635882309F082C0F0E0EE57FC4F20
:101ED000E4911E1708F04DC1E0916035882309F0A8
:101EE00074C0F0E0EE57FC4FE49180916235E89FBA
:101EF000802D1124810F80938B3790E0DC01A15954
:101F0000B84C2C9122FDE0C0982F8827990F845A55
:101F10009A4F90933505809334058C9184608C930F
:101F20008C918D7F8C9380916035809387378091E1
:101F3000623580938837109389372B9810928E37AB
:101F400010928D3710928C37809132059091330525
:101F5000019661CF50918A37452F407C4E2B2091BE
:101F60008C3742278431910578F0E0913405F09167
:101F700035054193F0933505E093340550918A3748
:101F8000809132059091330560918F3720918D3784
:101F900030E0260F311D240F311D20938D373093F3
:101FA0008F37550F550F50938A37019634CFEE0F68
:101FB000EE0FE0938A3780EC92E02DCF20913F0521
:101FC000222309F0F7CE019626CFE2E18ECFE2E19F
:101FD00080CF80918A37982F990F990F90938A37E5
:101FE000807C8E2B90918C37891709F46AC086E12A
:101FF00095E068E172E046E150E00E94C44A8EE359
:1020000090E090932F0580932E051092300581E08B
:102010008093643580932D0581E090E0FCCE509153
:102020008A37452F407C4E2B20918E3742278431B2
:10203000910578F0E0913405F09135054193F093E6
:102040003505E093340550918A378091320590919F
:10205000330560918F3720918C3730E0260F311D8A
:10206000240F311D20938C3730938F37550F550F28
:1020700050938A370196CFCE40918A374E2B2091CC
:102080008D3742278431910568F0E0913405F09155
:1020900035054193F0933505E09334058091320581
:1020A0009091330550918F3720918E3730E0250F76
:1020B000311D240F311D20938E3730938F370196B9
:1020C000AACE81EC92E0A7CE3091603520916235A6
:1020D0008DB79EB70C970FB6F8949EBF0FBE8DBFFD
:1020E000ADB7BEB7119686E195E0EDB7FEB7928326
:1020F000818386E190E013969C938E93129784E0FF
:1021000092E015969C938E93149716963C9316978F
:1021100017961C92179718962C93189719961C923D
:1021200019971A961C931A971B961C920E94D34AD1
:102130008DE390E090932F0580932E05109230054B
:1021400081E08093643580932D05109233051092C1
:10215000320580918B3790E02DB73EB7245F3F4F1B
:102160000FB6F8943EBF0FBE2DBFDC01A159B84C8D
:10217000CBCE209160358DB79EB70A970FB6F894F5
:102180009EBF0FBE8DBFADB7BEB7119686E195E07D
:10219000EDB7FEB79283818386E190E013969C931E
:1021A0008E9312978EEE91E015969C938E931497D2
:1021B00016961C93169717961C92179718962C93A1
:1021C000189719961C920E94D34A8CE390E0909342
:1021D0002F0580932E051092300581E080936435A1
:1021E00080932D051092330510923205809166354B
:1021F0002DB73EB7265F3F4F0FB6F8943EBF0FBED8
:102200002DBF6ACE80918A37982F990F990F90939E
:102210008A37807C8E2B90918D37891759F086E113
:1022200095E06BE272E046E150E00E94C44A8FE321
:1022300090E0E7CE82EC92E0EECD40916735509190
:102240006835E8E3F5E02591349160E07FEF2627DB
:10225000372791EA692F632770E0660F771F64586C
:102260007B4FFB0165917491322F22272627372758
:102270009327E92FF0E0EE0FFF1FE458FB4F659125
:102280007491322F222726273727EBEFE327F0E040
:10229000EE0FFF1FE458FB4F65917491322F2227F8
:1022A00026273727B82FBB0FA0E0A45ABA4F80E0EB
:1022B00090E0722F6627ED91E327F0E0EE0FFF1F0D
:1022C000E458FB4F2591349126273727019662E089
:1022D0008030960771F73093683520936735421741
:1022E0005307C9F086E195E061E572E046E150E010
:1022F0000E94C44A86E490E090932F0580932E05B7
:102300001092300581E08093643580932D05109202
:1023100033051092320508951F920F920FB60F9257
:102320000BB60F9211242F933F934F935F936F93AC
:102330007F938F939F93AF93BF93EF93FF9380917E
:1023400040058823D1F590B180913005882311F1A3
:10235000892F8078909131058917E1F080933105BC
:1023600090916635992309F440C0882399F120B1F2
:102370002F7080918A37282B20938A3780913205DD
:102380009091330582309105D9F0009781F5213A7B
:1023900009F45CC0FF91EF91BF91AF919F918F9134
:1023A0007F916F915F914F913F912F910F900BBE55
:1023B0000F900FBE0F901F9018950E94E81DEACF56
:1023C0002B3F09F45AC0213A29F310923305109299
:1023D0003205E0CF80B190E082959295907F98276A
:1023E000807F982780938A37D5CFCFDCD3CF8130B9
:1023F000910509F46FC032E08330930770F1A2E0D9
:1024000083309A0709F470C0B2E084309B0711F65C
:1024100030E08091673590916835822B932B9093B3
:1024200068358093673580918B3707DFE0918B3774
:10243000F0E0E159F84C8081826080838081816086
:10244000808380818B7F80832B9ABFCF81E090E057
:1024500090933305809332059DCF30918B37F32FC6
:10246000FF0FE0E0E80FF91FE75AFA4F20830196CB
:1024700090933305809332058DCF83E090E0909365
:1024800033058093320520916A3520938B37822F54
:1024900090E0FC01E159F84C308132FD30C0982FBA
:1024A0008827990F845A9A4F909335058093340565
:1024B00080818460808380818D7F8083809160357E
:1024C000809387378091623580938837209389374E
:1024D0002B9860CF213A09F078CF82E090E090937A
:1024E00033058093320556CF1092673520936835B7
:1024F00084E092E090933305809332054BCF509166
:102500006035409162352DB73EB72C5030400FB644
:10251000F8943EBF0FBE2DBFEDB7FEB7319626E152
:1025200035E0ADB7BEB712963C932E93119726E1D6
:1025300030E03383228324E032E0358324835683E2
:10254000178240871186938782870E94D34A87E447
:1025500090E090932F0580932E051092300581E036
:102560008093643580932D051092330510923205C7
:102570002DB73EB7245F3F4F0FB6F8943EBF0FBE56
:102580002DBF08CFF89490913005992341F48F77AF
:1025900082B9459A079BFECF0799FECF459878945C
:1025A00008958AE082B9459A079BFECF0799FECF2E
:1025B0004598E091683581EAE827F0E0EE0FFF1FCB
:1025C000E458FB4F859194913091673520E0822744
:1025D0009327909368358093673581E182B9459A56
:1025E000079BFECF0799FECF45980895982F9295A7
:1025F0009F7092B9459A079BFECF0799FECF4598E9
:10260000482F4F70E0916835E827F0E0EE0FFF1F8C
:10261000E458FB4F859194913091673520E08227F3
:102620009327909368358093673542B9459A079B05
:10263000FECF0799FECF459808952F923F924F9273
:102640005F926F927F928F929F92AF92BF92CF9242
:10265000DF92EF92FF920F931F93DF93CF9300D0FF
:102660000F92CDB7DEB78983692EA5E2CA2EA3E00B
:10267000DA2E992422243324EE24FF2400E010E0F3
:1026800088C01070C801880F991F2801440C452C80
:10269000441C55085194482A592AF6010191852D68
:1026A0009927820D931D800F911DAFEF4A2255246B
:1026B000D6011196AC906F010894C11CD11CA701E2
:1026C0004A0D511D9C0120703170232F3327420F7A
:1026D000531F3FEF232E312C2822392271802FEFF8
:1026E000E22EF12CE422F522872C8E24042510E022
:1026F000A224BB24F501E07CF070F595E795F595F3
:10270000E795F595E795F595E7959801207C30706C
:102710003595279535952795E22BF32B882D8295B6
:1027200086958695837090E0E82BF92BEE52FC4F4E
:1027300084914A835B8326DF0F7310700E521C4F07
:10274000F80184911FDF809164354A815B81882381
:1027500009F0A9C00894C11CD11C8201070D111DEC
:1027600040705170452F5527040F151FF501EF7369
:10277000F070EE52FC4F849105DFE82DF0E0EF732E
:10278000F070EE52FC4F8491FDDE9394F92DFE3AE9
:1027900041F0292D243009F074CF9981C92ED62C0F
:1027A00070CF1070C801880F991F5801AA0CAB2C6C
:1027B000AA1CBB08B194A82AB92AD6010C91200EF4
:1027C000311C8B2D9927280E391E1196CC90EC0CBC
:1027D000F11CC10180709170892F9927E80EF91EB4
:1027E0000A2510E0C224DD24F601E07CF070F595A6
:1027F000E795F595E795F595E795F595E795C80182
:10280000807C90709595879595958795E82BF92B09
:10281000EE52FC4F8491B6DEF801EF73F070EE5289
:10282000FC4F8491AFDEF601EF73F070EE52FC4F77
:102830008491A8DEF101E07CF070F695E795F695BD
:10284000E795C501807C90700024880F991F001CBB
:10285000880F991F001C892F902DE82BF92BC70199
:10286000807C9070929582958F7089279F708927C0
:10287000E82BF92BEE52FC4F849184DEF101EF73CB
:10288000F070EE52FC4F84917DDEF701EF73F07033
:10289000EE52FC4F849176DEF501EF73F070EE524C
:1028A000FC4F84916FDE0F900F900F90CF91DF91CE
:1028B0001F910F91FF90EF90DF90CF90BF90AF905E
:1028C0009F908F907F906F905F904F903F902F9050
:1028D00008951F930E94C02F80E060E00E946D2E3B
:1028E00086EC97E360E044E50E94942E80E061E08E
:1028F0000E946D2E81E495E060EB77E343E00E9457
:10290000103B882309F48AC08091DC37833029F199
:10291000863019F182E08093693581E495E067E3C0
:1029200075E04BE355E00E9432348823D1F48DE109
:1029300097E060E00E94152F8FEF93E2A4EF8150A3
:102940009040A040E1F700C0000010E081E495E075
:102950000E940F38812F1F91089581E0809369357F
:10296000DCCF80E061E00E946D2E8091DC37853005
:1029700009F4BFC0863008F05FC0833009F4A1C0FD
:10298000843039F48FEF96E060E00E94152F80913B
:10299000DC3791E0863008F490E090936E374F99E1
:1029A0008CC0992309F45CC081E080933F0548E71F
:1029B00054E060E070E081E495E00E94273781E414
:1029C00095E06CE575E040E052E00E94A535E091AD
:1029D0005C05F0E0E35AFA4F10821092720580E035
:1029E00062E00E946D2E8DE595E060E044E50E9476
:1029F000942E80E064E00E946D2E84EA96E060E010
:102A00000E94152F80913F05882379F511E081E41C
:102A100095E00E940F38812F1F91089581E495E081
:102A200060EB77E341E00E94103B882309F464C027
:102A300081E080933F0571CF873009F452C0873021
:102A400008F447C0883009F0A4CF82EB96E060E03C
:102A50000E94152F81E0809366358091DC3799CFF5
:102A600044E254E060E070E0A6CF8DE460E00E94B4
:102A70006D2E81E060E00E945E2E81E068E70E949A
:102A80005E2E81E06EE70E945E2E81E069E70E9483
:102A90005E2E81E069E70E945E2E81E06EE70E9473
:102AA0005E2E81E068E70E945E2E11E081E495E0F1
:102AB0000E940F38812F1F91089581E080933F0578
:102AC00070CF8EE097E060E00E94152F8091DC3798
:102AD00060CF8BED96E060E00E94152F8091DC378F
:102AE00058CF87EC96E060E00E94152F8091DC378C
:102AF00050CF8FEE96E0ABCF81E397E060E00E948D
:102B0000152F1ACF28988FE798E3A1E081509040C5
:102B1000A040E1F700C0000082E282B95D98289AE7
:102B20000C94CC2F559A209A3A9A3D9A3E9A3B9A09
:102B3000239A289A429A45984698439A2B9A8FE767
:102B400081B95C9A599A5A9A5F9A5B9A179A589ADD
:102B5000409A419AE3E7F0E0808181608083EDE66E
:102B6000F0E080818260808380818160808308952D
:102B70001F931FB7F894D6DF10926035109261351D
:102B800010926435109262351092633510923005C0
:102B90001092653582E08093693510926A35109203
:102BA0003F051092663510922D0510923605109251
:102BB0006D3510922F0510922E051092330510924C
:102BC000320580E090E0FC01E159F84C108201965A
:102BD00088319105C1F711B8469A28988FE798E394
:102BE000A1E081509040A040E1F700C0000080B11A
:102BF0008F7780932C0546988FE781B9289A82DFDA
:102C00000E94C02F1FBF1F910895E4E6F0E080816D
:102C1000877F808383E48093800089E180938100B3
:102C20000C941D0D909166359923E1F4E82FF0E0A6
:102C3000EE57FC4FE491F0E0262F30E02E173F07CF
:102C4000B4F4AF014F5F5F4F55954795E0FD14C059
:102C500031972E173F0759F06417B0F0862F8F5F1A
:102C6000841B0895262F30E02131310514F080E0D7
:102C70000895862F8F5F0895E42FF0E031972E1787
:102C80003F0751F780E00895842F860F0895FF9243
:102C90000F931F938C01F22E0E943131882379F11A
:102CA000C8016EE675E30E948930882399F1E2EC51
:102CB000F5E3BF2DBB0FA0E0A45ABA4F81918D93CD
:102CC00087E3EE36F807D1F7C8016EE675E30E9498
:102CD0008930882321F1EEE6F5E3BF2DBB0FA0E09C
:102CE000A85FB84F81918D9385E3E23CF807D1F757
:102CF000C8010E9419311F910F91FF9008958FE52F
:102D000092E00E943F05C8016EE675E30E9489309B
:102D1000882369F683E792E00E943F05C8CF83E7E6
:102D200092E00E943F05D7CF2F923F924F925F9241
:102D30007F928F929F92AF92BF92CF92DF92EF924B
:102D4000FF920F931F93DF93CF93CDB7DEB76097BA
:102D50000FB6F894DEBF0FBECDBF982E792E862E0B
:102D600080916635882309F4BAC004E210E082E15C
:102D7000482E512C80E090E020E0FF24B8E1EB2EBB
:102D8000A6E1AA2EB12CF3E8CF2EF2E0DF2E180137
:102D9000122F8159984CDC018C9180FF36C08091B4
:102DA0008737881669F1809187372DB73EB72A504B
:102DB00030400FB6F8943EBF0FBE2DBFEDB7FEB743
:102DC000319626E135E0ADB7BEB712963C932E930F
:102DD0001197B382A282D582C482868217828087AD
:102DE00011860E94D34A4DB75EB7465F5F4F0FB65C
:102DF000F8945EBF0FBE4DBF86E195E00E943F058F
:102E00005E2D583109F468C0F12E1F5F812F90E0CC
:102E1000821593050CF45CC0BE2DB83109F440C096
:102E200080913F05882361F468C0EE2DF0E0E15900
:102E3000F84C80818E7F808380818B7F8083E394B8
:102E4000FE1498F7EDB7FEB738970FB6F894FEBFAB
:102E50000FBEEDBF319606E115E0ADB7BEB71296D5
:102E60001C930E93119786E190E09383828388E907
:102E700092E095838483868217820E94D34AEDB7BD
:102E8000FEB738960FB6F894FEBF0FBEEDBF80E0D8
:102E900065E00E946D2EC80160E044E50E94942E1A
:102EA00060960FB6F894DEBF0FBECDBFCF91DF9115
:102EB0001F910F91FF90EF90DF90CF90BF90AF9058
:102EC0009F908F907F905F904F903F902F900895AC
:102ED000183109F4A1CF5DCFF12EE12E96CFE62F68
:102EE000F0E0EE57FC4FE4914E2E55248201000F86
:102EF000111F01151105A1F23DCF0E94262E0E943F
:102F0000522E6B877C878D879E87FE1408F467C1DD
:102F1000482D50E05A8749871A01220C331CC10101
:102F2000880F991F880F991F880F991F820D931D75
:102F30009C0140E050E029833A834B835C830E2D53
:102F4000F101EE51FD4F859194919C0140E050E0DC
:102F50002D833E834F8358871E2DAF2C42C0809017
:102F600088372091693530E040E050E069817A810E
:102F70008B819C810E94E6496B017C018091370521
:102F800090913805A0913905B0913A05C80ED91E27
:102F9000EA1EFB1E282D30E0429EC001439E900D8C
:102FA000529E900D1124AA2797FDA095BA2FC80E06
:102FB000D91EEA1EFB1EC00ED11CE11CF11C2F8580
:102FC0003889322F2227330F245A3A4F892D972DD3
:102FD000B701A6010E945131882371F10F5FA0163D
:102FE00090F1402F50E0588B4F87FA01E159F84C8F
:102FF000808180FDF3CF80916635882309F0AFCFC3
:10300000C0903705D0903805E0903905F0903A052A
:10301000C00ED11CE11CF11C2091693530E040E06C
:1030200050E06D817E818F8198850E94E649C60EB1
:10303000D71EE81EF91EC3CF8DEA92E00E943F051D
:103040000F5FA01670F6E12EFA2C8091663588236A
:1030500009F050C0F101EE51FD4F65917491A090BF
:103060003705B0903805C0903905D0903A05AE0CC0
:10307000B11CC11CD11C80E090E02091693530E08A
:1030800040E050E00E94E649A60EB71EC81ED91EB9
:103090000F2D10E00F5F1F4F0E191109222717FD8A
:1030A0002095322F892D972DB601A5010E94EC3273
:1030B000882359F48AC0F801E159F84C80818E7F49
:1030C000808380818B7F8083E394FE14D8F10E2D62
:1030D00010E0B801762F6627770F645A7A4F892D52
:1030E000972D0E947A32882331F780ED92E00E947A
:1030F0003F05E1CF8091883790E0489E5001499E7E
:10310000B00C589EB00C1124CC24B7FCC094DC2C1D
:103110008091370590913805A0913905B0913A0515
:10312000A80EB91ECA1EDB1EAE0CB11CC11CD11CE0
:10313000B101660F771F660F771F660F771F620D4D
:10314000731D99CF892D972D0E942D33882309F463
:1031500041C089E1809336050E942A2E0E94522E9A
:10316000ADB7BEB71C970FB6F894BEBF0FBEADBFCC
:10317000EDB7FEB7319606E115E012961C930E935B
:10318000119726E130E03383228321EF32E035834B
:10319000248329853A85378326832B853C854D8575
:1031A0005E85621B730B840B950B6087718782872A
:1031B00093870E94D34A4DB75EB7445F5F4F0FB607
:1031C000F8945EBF0FBE4DBF62CE8DEB92E00E94C1
:1031D0003F057BCF8FED92E00E943F05BACF282DAF
:1031E00030E03A8729871901220C331C2ECF2F9209
:1031F0003F924F925F926F927F928F929F92AF9287
:10320000BF92CF92DF92EF92FF920F931F93DF93C3
:10321000CF93CDB7DEB762970FB6F894DEBF0FBE7F
:10322000CDBF8C010E94692AC8010E947C2C96E1C6
:10323000A92E95E0B92E4424552486E1282E312C60
:103240001A8B098B80912D058823E1F5F894F09075
:103250006035E090623510926435789480916535E0
:10326000882309F088C009891A89809164358823E8
:1032700019F54B9B04C0079975C0F201099549994E
:1032800026C08091AE379091AF37009771F30197C8
:103290009093AF378093AE37C8010E947C2C8FEF9C
:1032A00094E3ACE081509040A040E1F700C0000002
:1032B000809164358823E9F21A8B098B80912D0562
:1032C000882321F286E195E00E943F05BFCF4A9B0B
:1032D00043C04C99CACF1A8B098B8091DC3781305F
:1032E00009F49DC2823009F42CC280916800886084
:1032F000809368008091680084608093680080916A
:103300006800846080936800809168008160809389
:103310006800109260350E94C02FDBDA882309F420
:1033200091CF80913F0591E089279091663599234F
:1033300009F4826082B9459AA7E8B3E11197F1F7E1
:1033400000C000004598B2E4BA95F1F700C0429879
:10335000E1E0E093653576CF8091AE379091AF375D
:10336000019696CF89B180FF88CF86B180FF85CF47
:10337000319985CF82CF0F2D10E02DB73EB7285061
:1033800030400FB6F8943EBF0FBE2DBFEDB7FEB76D
:103390003196ADB7BEB71296BC92AE9211973382FA
:1033A0002282B9E06B2EB3E07B2E75826482178394
:1033B00006830E94D34A2DB73EB7285F3F4F0FB612
:1033C000F8943EBF0FBE2DBF88E164E00E946D2ED1
:1033D000C50160E044E50E94942ECE2CDD248DB71B
:1033E0009EB708970FB6F8949EBF0FBE8DBFEDB77E
:1033F000FEB73196ADB7BEB71296BC92AE9211979A
:1034000033822282AEE06A2EA3E07A2E7582648235
:10341000D782C6820E94D34A2DB73EB7285F3F4F5E
:103420000FB6F8943EBF0FBE2DBF88E364E00E9444
:103430006D2EC50160E044E50E94942E80916135B7
:103440008F1509F45AC16091613589899A896CDCBC
:10345000F0926135E092633580E090E049895A89C5
:10346000FC01E159F84C20812D7F208301968831A1
:103470009105B1F75A8B498B4A01809164358823B5
:1034800009F036C180913005882309F01FC13F2D16
:10349000303598F79A8A898A80916635882309F0B1
:1034A0004EC1F801EE57FC4F249180916A35821786
:1034B00010F010926A3586B14B9990C2881F882708
:1034C000881F89832E9D902D11249D83A801440F70
:1034D000551FCA01880F991F880F991F880F991FC0
:1034E000840F951F8A879B8730E02C9DC0012D9DFE
:1034F000900D3C9D900D11243C01882477FC809414
:10350000982C6E827F8288869986002E012F000C6F
:10351000001F110B000C001F111FCC0CDD1CC294EE
:10352000D29460EFD622DC24C622DC24702E7C28C4
:103530007A82872D90E08E529C4F4E515D4FFA015A
:10354000859094909D868C862F2D2F732B83E22F50
:10355000F0E0EE52FC4F34913E87FC01F491FF877E
:10356000FC82E88A69887A8816B11095111F1127A4
:10357000111F09F420C18980811671F080E464E094
:103580000E946D2E112309F41AC188E996E060E0CB
:103590000E94152F21E0298380913605813009F49E
:1035A00015C180916635882309F4C4C000916A353D
:1035B000F894802E9924C4018159984C9A8B898B58
:1035C000DC018C9181FD97C08C9182FD94C08C911F
:1035D00084608C9381E07894882309F440C08091C2
:1035E0006635882309F011C16C857D8580916A3527
:1035F000C0903705D0903805E0903905F0903A0535
:10360000C80ED11CE11CF11C8E819F81A885B98553
:10361000C80ED91EEA1EFB1E80E090E0209169359D
:1036200030E040E050E00E94E649C60ED71EE81E9A
:10363000F91E0E94262E80916E37882309F4D2C08D
:10364000C301B701A601202F22DB0E942A2EA989DF
:10365000BA898C9182608C938C918B7F8C938091B2
:103660006A35882301F5112359F085B1B8E08B271D
:1036700085B980913605823018F0815080933605E7
:1036800020916D35275E20936D352D3708F0C2C02F
:1036900030E080916B3590916C35821B930B909349
:1036A00089008093880080916635882391F112E328
:1036B00006C08EE40E94F612115009F4AAC180914E
:1036C00064358823B1F37A8A698ABCCD80E464E0EA
:1036D0000E946D2E8EE996E060E00E94152F809189
:1036E00064358823E1F380916435882309F4CACED8
:1036F0009A8A898AA7CD80E06ECF8091663588232B
:1037000029F0809163358E1509F09DCE89889A88BD
:10371000B4CE00E010E009C08FEF0E94C2120F5F2C
:103720001F4F0733110509F493C080916435882336
:1037300099F3C9CF00916A353D81030F39CF22E15A
:10374000B4CE8091DD3781508093DD3789899A89A5
:1037500061E00E94183B8091DD378823A1F010E0E2
:10376000E988FA889DE0199FB0011124645A7C4CC5
:10377000C70141E00E94363B1F5F8091DD3718177B
:1037800088F3FA8AE98A1092AF371092AE370E9416
:10379000C02F89899A890E94692A89899A890E94F9
:1037A0007C2C8FEF99E6A8E181509040A040E1F792
:1037B00000C0000047CDC3016C81B6DADCCE82E9DF
:1037C00096E060E00E94152F2B9A19821092360520
:1037D00080E065E00E946D2E8CE796E060E00E943C
:1037E000152FDFCE9401322F2227330F245A3A4F60
:1037F000C301B701A6010E945131882309F025CFEA
:1038000082E193E00E943F0520CF9A858B85692F46
:10381000782FECCE10926D3520E030E03ACF109149
:10382000DD37ADE01A9FC0011124845A9C4C60EB37
:1038300077E34DE050E00E94C44A1F5F1093DD37EC
:1038400089899A8960EB77E341E00E94363B9BCF00
:10385000E7E5F2E03197F1F700C0000080916935AB
:10386000823009F436C112E000916A3580916435E6
:10387000882309F028CF85ED0E94C212809164351B
:10388000882309F020CF8AEA0E94C2128091643511
:10389000882309F018CF86E90E94C212809164350E
:1038A000882309F010CF8E850E94C2128091643562
:1038B000882309F008CFE0916A35F0E0EE52FC4F22
:1038C00084910E94C21280916435882309F0FBCE56
:1038D0008F850E94C21280916435882309F0F3CE4F
:1038E000E12FF0E0EE52FC4F84910E94C2128091D1
:1038F0006435882309F0E7CEEB81E027FA81EF27D2
:10390000E127EF73F0E0EE52FC4F84910E94C21267
:1039100080916435882309F0D6CE8EED0E94C212C4
:1039200080916435882309F0CECE8AEA0E94C212C3
:103930008FEC97E00197F1F700C0000080916435AB
:10394000882309F0C0CE85ED0E94C21280916435B3
:10395000882309F0B8CE8AEA0E94C21280916435A9
:10396000882309F0B0CE8DEA0E94C212809164359E
:10397000882309F0A8CEE0916A35F0E0EE52FC4FC2
:1039800084910E94C212C401982F8827990F845AEB
:103990009A4F0E941D1380916435882309F093CEBD
:1039A0008EED0E94C21280916435882309F08BCE7F
:1039B0008AEA0E94C21280916435882309F083CE7E
:1039C0008FEF0E94C2128C8160916A352BD980934F
:1039D0006A354B9BC9CDFC807A8A698A4598429AA0
:1039E0001092653589899A896F2D9ED98FE79AE162
:1039F000A6E081509040A040E1F700C00000B8D898
:103A000089899A890E94692A89899A890E947C2CCD
:103A100019CC1CE080916435882309F054CE0E94B3
:103A2000F6121150B9F7EFEFFFEFF0936835E0931E
:103A300067350E94D1120E94D1120E94D11280914A
:103A40006435882309F03FCE8EEF0E94F6128091F4
:103A50006435882309F037CE8C810E94F61280915C
:103A60006435882309F02FCE88890E94F612809150
:103A70006435882309F027CE80916A358F5F0E94D4
:103A8000F61280916435882309F01DCE82E00E94F1
:103A9000F6121091673580916835909164359923BD
:103AA00009F011CE0E94F61280916435882309F046
:103AB0000ACE812F0E94F61210E006C08EE40E940A
:103AC000F6121F5F163139F0809164358823B1F307
:103AD000FACD12E2C9CE10E080916435882309F056
:103AE000F2CD0E94F6121F5F1C30B1F72FEF3FEFAF
:103AF00030936835209367350E94D1120E94D1120D
:103B00000E94D11280916435882309F0DCCD8BEFBF
:103B10000E94F6128401102F0027110F045A1A4F29
:103B200080E090E07C010AC00E94F6120894E11C3B
:103B3000F11CB0E0EB16B2E0FB0641F0D8018D912C
:103B40008D0190916435992379F3BDCD109167353E
:103B50008091683590916435992309F0B4CD0E9425
:103B6000F61280916435882309F0ADCD812F0E9433
:103B7000F61229CF429A089590913005981789F04E
:103B80008093300580913005882361F48FE781B9F7
:103B9000469880916B008F7780936B0081E08093D3
:103BA0009237089511B8469A80B180788093310594
:103BB00010923305109232051092A9371092A8374F
:103BC0001092A73780916B00806880936B000895F6
:103BD0001F9390B180919037882309F040C090786E
:103BE000809131059817D9F1909331058091320574
:103BF0009091330583309105A0F1AC0143505040C2
:103C000020919537309196374217530741F110B103
:103C100010682091A737222339F09C01277030705B
:103C20002330310509F44FC00097B1F5163961F121
:103C300022E08D36920708F066C0E0913405F091DD
:103C400035051193F0933505E093340580913205E5
:103C500090913305019690933305809332051F911F
:103C6000089510B110680097A1F61A3A91F216392A
:103C700081F28091A8379091A93701969093A93746
:103C80008093A8371F9108958BE393E00E943F052E
:103C9000809132059091330581309105C9F4113836
:103CA00048F1115810939437212F30E02F5F3F4F88
:103CB000220F331F220F331F220F331F30939637EB
:103CC00020939537C7CF1A3A51F61092A737C7CF2E
:103CD0008230910509F0ACCF1138F0F011581093F3
:103CE00097372091A0373091A13730933505209335
:103CF0003405B0CF85E493E00E943F058091320502
:103D000090913305CECF8FE593E00E943F058091DF
:103D10003205909133059ECF80E593E00E943F05E8
:103D20008091320590913305D9CF86B1881F8827BD
:103D3000881F489B28C022E04B9B23C094E0820F41
:103D4000890F382F0FC022E04B9B18C094E0820FE0
:103D5000890F831729F08230C1F08430C1F0382FE9
:103D6000813071F096B190FDFBCF86B1881F882716
:103D7000881F4899E8CF20E04B99E8CF90E0E7CF43
:103D8000089590E0DCCF20E0D7CF80E0089580E078
:103D90000895F89490919037913011F078940895A7
:103DA0008F7782B9459A079BFECF0799FECF45983A
:103DB000789408951F93CF93DF938AEAEADF809186
:103DC000A4379091A537009709F444C0C0E0D0E033
:103DD0001AC012E04B9B27C094E0180F190F39F15D
:103DE000113009F03EC0E091A037F091A137EC0FFF
:103DF000FD1F8081CEDF21968091A4379091A53759
:103E0000C817D90738F5CE0187709070009759F719
:103E1000309916C086B1881F8827881F4899D9CF46
:103E200010E04B99D9CF90E0180F190FC9F67DDF3C
:103E3000882309F447C080E0ACDF8AEAAADFD3CF49
:103E400080E065E00E946D2E8FEB98E060E00E94BC
:103E5000152FFFCF80E09DDF81E0DF91CF911F9193
:103E6000089580E065E00E946D2E8DB79EB708979B
:103E70000FB6F8949EBF0FBE8DBFEDB7FEB731965B
:103E8000C6E1D5E0ADB7BEB71296DC93CE931197DD
:103E900086E190E09383828387E693E09583848331
:103EA000168317820E94D34A8DB79EB708960FB625
:103EB000F8949EBF0FBE8DBFCE0160E044E50E9426
:103EC000942EFFCF80E0C9CF1F93CF93DF93182F9D
:103ED000EB01CB0167E070E00E94114A9B01220FC9
:103EE000331F220F331F220F331F261B370B2C17B4
:103EF0003D0721F08DE793E00E943F052091A23716
:103F00003091A337812F90E04DE152E0849FB001C2
:103F1000859F700D949F700D1124A901460F571FA6
:103F2000C60FD71FC20FD31FA091A037B091A137E2
:103F30004C175D0709F46DC0FA014DC080E0218186
:103F400030E03595279511962C931197918190FD2E
:103F50008068228130E03595279512962C93129730
:103F60008695928190FD8068238130E03595279574
:103F700013962C9313978695938190FD80682481E6
:103F800030E03595279514962C9314978695948157
:103F900090FD8068258130E03595279515962C9306
:103FA00015978695958190FD8068268130E035953E
:103FB000279516962C93169786959681379690FDA1
:103FC000806890E09595879517968C931797CE17F4
:103FD000DF0759F01896808190E0959587958C932E
:103FE000808180FFABCF80E4AACF495F5F4FC41BC5
:103FF000D50B88EB9DE6C89F9001C99F300DD89FD7
:10400000300D1124285F3F4FC901DF91CF911F91DF
:10401000089520E030E0F8CF0F931F93CF93DF9304
:1040200040919A3750E02DE132E0429FC001439F1A
:10403000900D529F900D1124C091A237D091A337BB
:10404000C80FD91F83E8888319821A821B821C82B9
:104050001D828E010A5F1F4F1F821E8281E090E049
:10406000F8019383828386EC848380913F058823C3
:1040700009F470C08EEC848380913B0590913C05DF
:10408000A0913D05B0913E0520913705309138054E
:104090004091390550913A05821B930BA40BB50B47
:1040A000F801A5839683878311861086138612866E
:1040B000ECE8F7E0D801A05CBF4F84918D93319676
:1040C00028E0EC38F207C9F784EB98E00E94884AB0
:1040D000F801E05CFE4F8083C8018F5B9E4F64EB6C
:1040E00078E04FE050E00E94914AFE01EA5AFE4F0C
:1040F00080E090E020E03991230F019631E0863591
:104100009307C9F72195208380919A3767E571E07D
:10411000DBDE9093A5378093A437E1E088389E07D3
:1041200089F089E893E00E943F058091A43790913F
:10413000A5379C01287F8217930721F089E993E036
:104140000E943F0537DE10929337DF91CF911F9188
:104150000F91089586EEF80184838ECF40919A37AF
:1041600050E02DE132E0429FC001439F900D529FED
:10417000900D1124E091A237F091A337E80FF91FB9
:1041800080E8808380919937818312821382148220
:104190001582DF01169680E090E01D920196843131
:1041A0009105D9F7DF01A65EBD4F80E090E020E0E9
:1041B0003191230F019632E08A319307C9F7219597
:1041C0002C9380919A376BE172E07EDE9093A53755
:1041D0008093A43722E08B36920708F03DC032E08E
:1041E0008836930789F089E893E00E943F05809123
:1041F000A4379091A5379C01287F8217930721F05F
:1042000089E993E00E943F05D5DD882311F12091D3
:10421000993721502093993780919C3790919D3701
:10422000A0919E37B0919F370196A11DB11D80933B
:104230009C3790939D37A0939E37B0939F3781E032
:10424000222319F080939337089580E08093933769
:10425000089510929337089589EA93E00E943F05EC
:104260008091A4379091A537BACF1F93182F409112
:104270009A3750E08DE192E0489F9001499F300DC0
:10428000589F300D1124E091A237F091A337E20F2F
:10429000F31F80919837805880838091993781836C
:1042A0001282138214821582DF01169620E030E01C
:1042B00080E09191890F2F5F3F4F26303105C9F77C
:1042C00081958C9380919A3767E070E0FDDD9C01C9
:1042D0009093A5378093A43782E02B36380798F562
:1042E0002830310589F089E893E00E943F058091EC
:1042F000A4379091A5379C01287F8217930721F05E
:1043000089E993E00E943F0555DD10929337112310
:10431000C1F08091993781508093993780919C3773
:1043200090919D37A0919E37B0919F370196A11D26
:10433000B11D80939C3790939D37A0939E37B09387
:104340009F371F91089589EA93E00E943F052091CD
:10435000A4373091A537C4CF80919837833091F03E
:10436000843038F08951823050F08AEB93E00C941D
:104370003F05882331F08130C1F781E076CF80E0BE
:1043800074CFECCE49CECF92DF92EF92FF920F9393
:104390001F93DF93CF9300D0CDB7DEB7C090320527
:1043A000D09033052DEF3FEFC20ED31EC114D104C0
:1043B00009F499C09601287F2C153D0509F4A2C087
:1043C00080E062E00E946D2E8DB79EB70C970FB60D
:1043D000F8949EBF0FBE8DBFEDB7FEB7319666E174
:1043E000E62E65E0F62EADB7BEB71296FC92EE92C1
:1043F000119786E190E0938382838EEC93E095831E
:104400008483809194378683178280919737808741
:104410001186D386C2860E94D34AEDB7FEB73C967A
:104420000FB6F894FEBF0FBEEDBFC70160E044E5D4
:104430000E94942E05E110E020E030E0802F8551AD
:1044400067E00E94054A492FC80167E070E00E94BA
:10445000254AFCE04F9F802D112429833A830E9436
:104460006D2E8DB79EB708970FB6F8949EBF0FBEFE
:104470008DBF4DB75EB74F5F5F4FADB7BEB71296FA
:10448000FC92EE92119786E190E0FA019383828389
:10449000A4EEB3E0B583A483A091A037B091A13777
:1044A00029813A81A20FB31F8C91868317820E94C3
:1044B000D34AEDB7FEB738960FB6F894FEBF0FBEDD
:1044C000EDBFC70160E044E50E94942E980124519D
:1044D00030402C153D0508F0FFCF0F5F1F4F08330C
:1044E0001105D1F3ABCF86EC93E00E943F050F900E
:1044F0000F90CF91DF911F910F91FF90EF90DF9080
:10450000CF900895E091A037F091A1372E0F3F1F73
:104510004091A2375091A337E217F30741F3682F78
:1045200070E08DE192E0689FD001699FB00D789FA7
:10453000B00D1124A40FB51F90818181880F492FE0
:104540004170842B8C939695492F41708281880FFE
:10455000842B11968C9311979695492F41708381E6
:10456000880F842B12968C9312979695492F417041
:104570008481880F842B13968C9313979695492FDB
:1045800041708581880F842B14968C931497892F02
:104590008695482F41709681990F942B15969C9380
:1045A000159790E09595879581709781990F982B35
:1045B00016969C931697179638962E173F0709F074
:1045C000BBCF95CFEF92FF920F931F93DF93CF93C3
:1045D00000D0CDB7DEB7109292378091A837909176
:1045E000A9378430910508F08BC0809132059091F5
:1045F0003305009709F483C080919A37C4DE209177
:1046000032053091330536952795369527953695A1
:104610002795C901880F991F880F991F880F991F27
:10462000821B930B2091A2373091A33760919A3768
:104630000097D1F0A62FB0E04DE152E0A49FF00129
:10464000A59FF00DB49FF00D1124E20FF31F40E081
:1046500050E070E0A1917A0F4F5F5F4F4817590704
:10466000C8F3772309F04CC1462F50E08DE192E06A
:10467000489FF001499FF00D589FF00D1124E20F63
:10468000F31F708170939837733009F42CC1743024
:1046900008F024C1772309F0BEC081818093993747
:1046A000828190E0A0E0B0E0DC0199278827238197
:1046B00030E040E050E0542F432F322F2227822B4E
:1046C000932BA42BB52B248130E040E050E0822BCB
:1046D000932BA42BB52B80939C3790939D37A0935D
:1046E0009E37B0939F3781E0809393370F900F9060
:1046F000CF91DF911F910F91FF90EF900895FFCF21
:1047000080E060E00E946D2E8DB79EB70A970FB6CD
:10471000F8949EBF0FBE8DBFEDB7FEB7319606E190
:1047200015E0ADB7BEB712961C930E93119786E1B4
:1047300090E0938382838AEE93E0958384838091D3
:10474000A8379091A93797838683809132059091FD
:104750003305918780870E94D34AEDB7FEB73A961A
:104760000FB6F894FEBF0FBEEDBFC80160E044E590
:104770000E94942EEE24FF2427E030E043C0C701BE
:10478000B9010E94114A6F5FFCE0F89F802D11244F
:1047900029833A830E946D2E8DB79EB708970FB676
:1047A000F8949EBF0FBE8DBFEDB7FEB73196ADB783
:1047B000BEB712961C930E93119786E190E09383F7
:1047C0008283ACEFB3E0B583A483A091A037B0910E
:1047D000A137AE0DBF1D8C91868317820E94D34AEC
:1047E000EDB7FEB738960FB6F894FEBF0FBEEDBF1B
:1047F000C80160E044E50E94942E0894E11CF11C7D
:104800003A8129818091A8379091A937E816F90655
:1048100008F4B5CFFFCF713009F47DC08091A63781
:1048200065E10E94054A682F6F5F892F880F880F06
:104830000E946D2E8FE30E94792E81E060E00E943D
:104840005E2E81E060E00E945E2E81E060E00E94CA
:104850005E2E8091A637883608F088C08F5F8093DF
:10486000A63780E065E00E946D2E8DB79EB70C974D
:104870000FB6F8949EBF0FBE8DBFEDB7FEB7319651
:1048800006E115E0ADB7BEB712961C930E931197D3
:1048900086E190E0938382838EE094E09583848325
:1048A000809198378683178280919437808711860C
:1048B00080919737828713860E94D34AEDB7FEB75F
:1048C0003C960FB6F894FEBF0FBEEDBFC80160E086
:1048D00044E50E94942E1092933708CF793108F462
:1048E0009DCF7B3120F481E080939337FFCE7134EC
:1048F00009F094CF81E08093983780939337F6CE78
:1049000081E094E00E943F052091A2373091A337C7
:1049100060919A37A9CE818180939937828190E006
:10492000A0E0B0E0DC0199278827238130E040E057
:1049300050E0542F432F322F2227822B932BA42B6E
:10494000B52B248130E040E050E0822B932BA42B48
:10495000B52B80939C3790939D37A0939E37B0934F
:104960009F3760939B3770939337C0CE1092A637D2
:1049700078CF0F931F93CF93DF9380E060E00E9486
:104980006D2EC2E2D4E081E495E0BE0143E00E94D6
:10499000103B882309F499C081E495E067E375E052
:1049A0004BE355E00E943234882381F480EA98E09A
:1049B00060E00E94152F8FEF93E2A4EF81509040AA
:1049C000A040E1F700C0000000E075C08CE898E06E
:1049D00060E00E94152F80E062E00E946D2EADB76E
:1049E000BEB71A970FB6F894BEBF0FBEADBFEDB7F6
:1049F000FEB73196C6E1D5E01296DC93CE931197BF
:104A000086E190E09383828389E394E095838483B5
:104A10008091520590915305A0915405B091550590
:104A200014E1B695A795979587951A95D1F7868342
:104A30009783A087B1870E94D34A8DB79EB70A9605
:104A40000FB6F8949EBF0FBE8DBFCE0160E044E567
:104A50000E94942E4F9B03C081E080933F0581E428
:104A600095E044E254E060E070E00E9427376091F6
:104A7000A2377091A33781E495E040E052E00E94B4
:104A8000A535E091A237F091A337EF0121968081FF
:104A9000FE01E80FF11D10821D8A80E061E00E9496
:104AA0006D2ECE0160E044E50E94942E80913F057A
:104AB0008823B9F401E081E495E00E940F38802F4B
:104AC000DF91CF911F910F91089581E495E0BE0190
:104AD00041E00E94103B882331F181E080933F0543
:104AE0005BCF8DE461E00E946D2E81E060E00E946A
:104AF0005E2E81E068E70E945E2E81E06EE70E94F4
:104B00005E2E81E069E70E945E2E81E069E70E94E7
:104B10005E2E81E06EE70E945E2E81E068E70E94D3
:104B20005E2E01E0C8CF8DB79EB708970FB6F894F8
:104B30009EBF0FBE8DBFEDB7FEB7319606E115E003
:104B4000ADB7BEB712961C930E93119786E190E015
:104B5000938382838BE294E095838483D783C68397
:104B60000E94D34A8DB79EB708960FB6F8949EBFA1
:104B70000FBE8DBFC80160E044E50E94942E1BCF9C
:104B8000CF92DF92EF92FF920F931F93DF93CF9319
:104B90000F92CDB7DEB76C01E0909C37F0909D3757
:104BA00000919E3710919F3780913705909138057D
:104BB000A0913905B0913A05E80EF91E0A1F1B1F96
:104BC00069830E94262E698170E02DE132E0629FA8
:104BD000C001639F900D729F900D11244A96209101
:104BE000A2373091A337280F391FC601B801A7019A
:104BF0000E945131882321F480E494E00E943F0513
:104C00000E942A2E0F90CF91DF911F910F91FF905C
:104C1000EF90DF90CF9008954F925F926F927F92C6
:104C20008F929F92AF92BF92CF92DF92EF92FF92BC
:104C30000F931F93CF93DF93E82E992E862EF42E99
:104C4000442E552466247724A0903705B09038056B
:104C5000C0903905D0903A0580919C3790919D374E
:104C6000A0919E37B0919F37A80EB91ECA1EDB1EB9
:104C70000894A11CB11CC11CD11CA418B508C608FD
:104C8000D708E4D78E2D992DB601A5019301820195
:104C90000E94EC32882309F44AC0FF2061F1182DEC
:104CA00000E0CDE1D2E006C01F5F143101F10F5FDB
:104CB0000F1508F5212F30E02C9FC0012D9F900D7E
:104CC0003C9F900D11244A966091A2377091A337B2
:104CD000680F791F8E2D992D0E947A32882321F733
:104CE00087E694E00E943F051F5F143101F710E052
:104CF0000F5F0F15F8F28E2D992D0E942D3388230A
:104D000021F489E794E00E943F05A4D7DF91CF9179
:104D10001F910F91FF90EF90DF90CF90BF90AF90D9
:104D20009F908F907F906F905F904F90089581E556
:104D300094E00E943F05B1CF80913F0591E0892723
:104D4000866046989FE791B982B9429A459A87E86A
:104D500093E10197F1F700C00000459892E49A951D
:104D6000F1F700C008958FE781B9559A209A3A9AD1
:104D70003D9A3E9A3B9A239A5C9A599A5A9A5F9A1C
:104D8000179A589A409A5B9A5D98289A429A459841
:104D90004698439A2B9A08951F931FB7F894E3DF20
:104DA00082E08093913710929037809190378823DA
:104DB00089F55D9810929337109230051092A737BD
:104DC00010923F051092360510923305109232056D
:104DD0001092923710929A3711B8469A28988FE716
:104DE00098E3A1E081509040A040E1F700C00000AE
:104DF00080B18F7780932C05289A80916400877FFB
:104E00008093640099DF0E94CC2F0E94C02F1FBFA7
:104E10001F9108955D9ACECFAF92BF92CF92DF924D
:104E2000EF92FF920F931F93DF93CF9300D0CDB7F4
:104E3000DEB75C018CE595E09093A1378093A037B5
:104E400086EC97E09093A3378093A23792DD882376
:104E500009F4FFCF71DF80916B008F7780936B0037
:104E6000809168008160809368000FEF86B180FDBB
:104E7000FDCF86B1881F8827881F489B48C022E045
:104E80004B9B48C094E0D22ED80ED90E80913005AD
:104E9000882321F0809191378130F1F180913005A4
:104EA000882311F180913205909133050097E1F04C
:104EB0002D2D2130C9F08330910540F48EE894E027
:104EC0000E943F0580913205909133052DEFE22E2F
:104ED0002FEFF22EE80EF91E8091953790919637BC
:104EE0008E159F0509F07DC080919137D81609F481
:104EF000BDCFFD2DF53008F0B9CFF230C9F1F33058
:104F000098F4F13009F44AC0D0929137AFCF20E045
:104F10004B99B8CF90E0B7CFDD2009F0BFCF809399
:104F2000A7370E94951EA2CF2D2D233079F0243073
:104F300059F780E00E94BC1D429A1092923710925D
:104F400093370093983710929A37DECF809193373A
:104F50008823D1F680919137823009F4FDC0809189
:104F60009137813089F680E00E94BC1D429ACCCFF7
:104F70002B9A429A80919237882309F023DB809103
:104F80009337882309F4C0CF80919837882309F498
:104F9000D3C0813009F4A5C04298B6CF2B98809138
:104FA00093378823C9F3809191374298D0929037F4
:104FB00080919037882309F092C05D98CDD91092E6
:104FC000903780919037882309F087C05D98429A86
:104FD00080919A378F5F80939A37843109F094CF0C
:104FE000B2CFADB7BEB71C970FB6F894BEBF0FBE19
:104FF000ADBFEDB7FEB7319606E115E012961C93F2
:105000000E93119726E130E03383228329E934E0BF
:1050100035832483D682178291878087F386E28640
:105020000E94D34AEDB7FEB73C960FB6F894FEBF88
:105030000FBEEDBF80E060E050D6C80160E044E5FF
:1050400073D6CC24DD2427E030E0CE14DF0408F052
:10505000FFCFFCE1CF16D104D9F3C601B9010E94FC
:10506000114A6E5F9CE0989F802D112429833A831A
:1050700034D6ADB7BEB718970FB6F894BEBF0FBE03
:10508000ADBFEDB7FEB7319612961C930E931197F4
:1050900086E190E093838283A4EEB3E0B583A4839A
:1050A000A091A037B091A137AC0DBD1D8C91868326
:1050B00017820E94D34AEDB7FEB738960FB6F89420
:1050C000FEBF0FBEEDBFC80160E044E52DD60894D9
:1050D000C11CD11C29813A81B8CF5D9A78CF5D9AE5
:1050E0006DCF80919937813071F170919A37872F08
:1050F00090E060919B37262F30E0A901415050404D
:105100008417950731F02D5E3F4F8217930709F002
:1051100043CF7617E8F0472F4F5F461BC5017CDD74
:1051200080919A378F5F80939B37843109F034CF19
:1051300010929B374298E8CEC50160919A3720DDE6
:105140008091983726CF70919A3760919B37E1CF45
:10515000472F4B5E461BE2CF81E00E94BC1D429868
:10516000D3CE2F923F924F925F926F927F928F9207
:105170009F92AF92BF92CF92DF92EF92FF920F93E6
:105180001F93DF93CF93CDB7DEB72D970FB6F8946B
:10519000DEBF0FBECDBF8B014A013E010894611CEA
:1051A000711CD301E6EDF4E02DE001900D92215049
:1051B000E1F7BB244424AA2452E8552E42E2E42E0F
:1051C000F12CE80EF91E3EE0C32ED12CCC0EDD1ED4
:1051D00022E8222E312C280C391CC701B80140E2EC
:1051E00050E00E94A53580329105A1F4D8011B96AC
:1051F0008C911B9790E09C012F7330702F303105FC
:1052000059F183FD23C0F8018081853E19F188237F
:1052100009F05AC0D4011C9280E02D960FB6F89484
:10522000DEBF0FBECDBFCF91DF911F910F91FF90D9
:10523000EF90DF90CF90BF90AF909F908F907F9036
:105240006F905F904F903F902F900895F80180816C
:10525000882301F3BB24C1CFBB2021F58C91982F6B
:10526000907E903409F0B9CF9FE1A92EA8221D9617
:105270004C90F1011082A5E7B0E085E7582EF301CC
:10528000AD01480D591D81919801280F311DD9019B
:105290008C91DA018D93AD01EC15FD05A1F7BB24CE
:1052A000B3949BCFD8018C91AA948A1599F61D9638
:1052B0008C911D97841571F6552009F48ECFB3EFAC
:1052C0005B0EA52DB0E0DBCF8E3221F2BB2081F04A
:1052D00031962BE090E001C08191392F379533272B
:1052E00037959695932B980F2150B1F7941531F07F
:1052F000C801B4010E94E53481E08FCFFA2DF1306E
:10530000B9F7452D50E043385105B4F79A0160E0F4
:1053100080E090E0880D991D280D391DD9012C9150
:10532000FC0120836F5F862F90E09C01240F351FC6
:10533000233831057CF381E070CFEF92FF920F9319
:105340001F93DF93CF93CDB7DEB7A9970FB6F8942D
:10535000DEBF0FBECDBFFC01DB018C918E32A9F107
:10536000838590E0887190708031910509F466C062
:10537000009759F5848D958DA68DB78D803020E4EA
:10538000920726E0A20720E0B20709F459C0803056
:1053900020E892072CE0A20720E0B20709F454C0ED
:1053A000803020E8920726E1A20720E0B20709F446
:1053B00049C081509044A640B0408F3F2FE29207F1
:1053C00021E1A20720E0B20778F020E0822FA99621
:1053D0000FB6F894DEBF0FBECDBFCF91DF911F9106
:1053E0000F91FF90EF900895CF017E010894E11C8A
:1053F000F11CB7010E94E5341E86198A8E01025FF6
:105400001F4FC801B70141E00E94103B882371F093
:10541000C8016EE675E340E052E00E94A535C80180
:105420000E940F388091C035813081F089898823AE
:1054300061F2C8010E940F3820E0C8CF21E0C6CF3A
:1054400023E0C4CF25E0C2CF24E0C0CF8091C13596
:10545000882361F78091AF3590E0A0E0B0E0BA2FEB
:10546000A92F982F88272091B035820F911DA11D5B
:10547000B11DB695A79597958795B695A7959795DC
:105480008795803921E0920720E0A20720E0B2074B
:10549000F1F0803223E0920720E0A20720E0B2077B
:1054A000A1F0803A25E0920720E0A20720E0B207B1
:1054B00009F0BCCF28E08989882309F487CFC80187
:1054C00029A70E940F3829A581CF27E0F4CF26E035
:1054D000F2CF2F923F924F925F926F927F928F9274
:1054E0009F92AF92BF92CF92DF92EF92FF920F9373
:1054F0001F93DF93CF93CDB7DEB7C05FD0400FB619
:10550000F894DEBF0FBECDBF7C011092AB37109276
:10551000AA37829640E050E0BA010E94273703E4A0
:10552000C02ED12CCC0EDD1E13E6A12EB12CAC0E5C
:10553000BD1EB4E26B2E712CC701B601A50111DEB0
:105540008823E1F18091AA379091AB3721E087342D
:10555000920708F0A7C1C601B501EFDE882E8823A7
:1055600059F38091AA379091AB37869D8001879D32
:10557000100D969D100D1124045A1A4FC801B50143
:1055800046E150E00E94C44AB8016A5E7F4FC601FE
:105590000E94E5348091AA379091AB37869DF00147
:1055A000879DF00D969DF00D1124E45AFA4F83A2C9
:1055B00001969093AB378093AA37BECF2091AA373C
:1055C0003091AB37C751DF4F39832883C95ED04054
:1055D000F70185A182508230A8F184E290E0C751A2
:1055E000DF4FE881F981C95ED040E89F8001E99FE3
:1055F000100DF89F100D1124045A1A4FC80162EBC8
:1056000074E046E150E00E94C44AC801469662EB4D
:1056100074E04DE050E00E94C44A82E0F80183A3A8
:10562000C751DF4F28813981C95ED0402F5F3F4F7E
:10563000C751DF4F39832883C95ED0403093AB37E1
:105640002093AA37AFE72A2EA5E03A2E80E090E01B
:105650007E010894E11CF11CF7E1CF2ED12CCC0E79
:10566000DD1EC751DF4FE881F981C95ED0408E173A
:105670009F0708F01EC1FC013196C351DF4FF9832B
:10568000E883CD5ED040C751DF4F28813981C95EA4
:10569000D040E217F30708F026C1C1018397F1015A
:1056A000B496C151DF4FF983E883CF5ED0405F01EC
:1056B000C351DF4F48805980CD5ED040CA51DF4F83
:1056C0008883C65ED04091012D503040C551DF4FD8
:1056D00039832883CB5ED040C951DF4F398228827D
:1056E000C75ED040392EC701CA51DF4F6881C65E00
:1056F000D040732D46E150E00E94C44A88240AC07D
:105700000E0D1F1DF801808190E00E94794AF8017A
:1057100080838394F70101900020E9F73197EE1917
:10572000FF09082D10E00E171F0750F3EDED8E2E28
:10573000EFEF9E2E8A0C9B1C682C292CC601B4010D
:1057400046E150E00E94C44A77240AC00C0D1D1D9A
:10575000F801808190E00E94794AF8018083739477
:10576000F60101900020E9F73197EC19FD09072DAA
:1057700010E00E171F0750F3C701B60146E150E0D5
:105780000E94B64A282F392FC951DF4FE881F9818D
:10579000C75ED04080818150823008F480C0F5011E
:1057A00080818150823008F477C0121613060CF005
:1057B00055C0CE018D96CA51DF4F6881C65ED0407C
:1057C000732D46E150E00E94C44ACA51DF4F8881E0
:1057D000C65ED040932D662D722D46E150E00E94AA
:1057E000C44A862D922DBE01635D7F4F46E150E095
:1057F0000E94C44ACE018D96C551DF4F68817981E0
:10580000CB5ED0404DE050E00E94C44A84010A5E65
:105810001F4FC551DF4F88819981CB5ED040B801C1
:105820004DE050E00E94C44AC801BE01635D7F4F55
:105830004DE050E00E94C44AC951DF4FE881F98130
:10584000C75ED0408081F5019081C951DF4FE8816A
:10585000F981C75ED0409083F50180830894411C94
:10586000511C24E230E0A20EB31EC751DF4F8881E5
:105870009981C95ED0404816590608F434CFC15109
:10588000DF4F28803980CF5ED040C351DF4F888101
:105890009981CD5ED040E5CE28513C4F86CF285E21
:1058A00033407DCFC751DF4F99838883C95ED04095
:1058B0008FCEC051DF4F0FB6F894DEBF0FBECDBF05
:1058C000CF91DF911F910F91FF90EF90DF90CF90DC
:1058D000BF90AF909F908F907F906F905F904F9010
:1058E0003F902F900895C1018496C151DF4F998355
:1058F0008883CF5ED040C3CF8F929F92AF92BF92EA
:10590000CF92DF92EF92FF920F931F93CF93DF938B
:105910008091AC379091AD372091AE373091AF3751
:105920002817390728F43093AD372093AC37C901D5
:1059300004968217930730F4245030403093AD37EB
:105940002093AC3780E060E0C8D181E06FE7B6D14A
:10595000C3E1D0E081E060E4B1D12197D9F785EBD4
:1059600094E0CBD2C3E1D0E081E060E4A7D12197FD
:10597000D9F781E06FE7A2D12091AA373091AB37F8
:105980002115310509F447C14091AC375091AD372D
:10599000CA0105964817590708F01EC14217530758
:1059A00008F01AC164E270E0469F7001479FF00C56
:1059B000569FF00C11248FE795E0E80EF91EEA01DE
:1059C00091E0C92ED12CBB24B3948091AE37909135
:1059D000AF37C817D90709F0BB24AC2C80E06C2D79
:1059E0007CD104E510E006C060E081E067D10150A1
:1059F000104041F0BB20C1F36FE781E05FD101505F
:105A00001040C1F781E06A2D68D187010352104030
:105A1000902E812EC8016B2D43E586D1F701808140
:105A20008150823008F4B7C0BB2009F09EC08601C7
:105A300021964091AC375091AD37CA010596C817F1
:105A4000D907C8F12091AA373091AB3726303105FC
:105A500008F044C0EE24E39482E56E2D3ED181E04F
:105A600060E02CD181E060E029D1E3947E2D763096
:105A700099F78091AC379091AD379801280F391F75
:105A80004091AE375091AF374217530708F4CBC05F
:105A9000215030403093AF372093AE37043011059A
:105AA00009F03ACF009709F437CF01979093AD37BB
:105AB0008093AC3731CF2091AA373091AB3708941F
:105AC000C11CD11C64E270E0E60EF71EC217D307BA
:105AD00008F479CF2630310508F4BCCFE7E2F0E0D6
:105AE0004E9FC0014F9F900D5E9F900D11248D53CE
:105AF0009F4FB9010E94114A88E0E82EE60E83EC20
:105B000090E0B9010E94114ACE2CC61AC8E0D0E03C
:105B1000BB24B39482E56B2DE0D081E060E0CED071
:105B20004C2F9E01295F3F4F2C173D070CF471C08D
:105B300060E00AC0E41650F0669560684F5F842FFD
:105B400090E0281739074CF04C15A0F766954F5F89
:105B5000842F90E028173907BCF781E0AFD0B394C9
:105B600028967B2D7630B1F684CF86EC97E3692DAD
:105B7000782D46E150E00E94C44AB8016A5E7F4F2A
:105B800080EB97E34DE050E00E94C44AF70180812A
:105B90008093DC374CCF89E46A2D9FD0BB20F9F08D
:105BA00081E06FE78BD081E063E488D081E06DE530
:105BB00085D081E06DE582D081E06DE57FD081E028
:105BC0006BE57CD081E06BE579D081E063E476D051
:105BD0006FE781E073D028CF00E010E037CF81E09D
:105BE00060E06CD081E06CE369D081E062E266D075
:105BF00081E062E263D081E062E260D081E064E251
:105C00005DD081E064E25AD081E06CE357D060E07F
:105C1000E0CF60E0A2CF80E061E05FD081EC94E073
:105C200060E044E581D0DF91CF911F910F91FF900B
:105C3000EF90DF90CF90BF90AF909F908F9008959E
:105C400014BC83E085BD81E085BB089581E080932D
:105C50006E00089510926E0008951F920F920FB675
:105C60000F9211248F939F93AF93BF938091DE3750
:105C70009091DF37A091E037B091E1370196A11DF7
:105C8000B11D8093DE379093DF37A093E037B09358
:105C9000E137BF91AF919F918F910F900FBE0F9001
:105CA0001F9018952FB7F8946091DE377091DF3709
:105CB0008091E0379091E1372FBF089590E59CBD2A
:105CC0001DBC882341F05E9A2A986EBD0DB407FE74
:105CD000FDCF2A9A08955E98F7CF1F93162F682F4D
:105CE000606880E0EBDF612F606480E0E7DF1F9198
:105CF00008950F931F93CF93DF9303E0809F80015C
:105D00001124E801C859D74F0559174FFE01649176
:105D1000660F81E0D3DF2196C017D107B9F7DF9175
:105D2000CF911F910F910895AF92BF92CF92DF92C2
:105D3000EF92FF920F931F93CF93DF93D62EC42E33
:105D4000E82EF92EBB248FE7A82EF70101917F01E1
:105D5000002359F4DF91CF911F910F91FF90EF90A5
:105D6000DF90CF90BF90AF900895BC1498F70D3698
:105D700009F183E0089F80011124E801C859D74F39
:105D80000659174FFE016491660FD1106A2581E014
:105D900095DFB394C017D10749F4BC14B0F6DD20E9
:105DA000C1F16FE781E08ADFB394CFCF2196BC14B5
:105DB00060F6E8CFDD2079F163E481E07FDFB39422
:105DC000BC1408F0C2CFDD2051F16BE781E076DF33
:105DD000B394BC1408F0B9CFDD2029F167E681E067
:105DE0006DDFB394BC1408F0B0CFDD20D1F06BE7C9
:105DF00081E064DFB394BC1408F0A7CFDD2069F024
:105E000067E481E05BDFB394BC1408F09ECFDD2033
:105E100041F660E0C7CF6CE3D0CF68E3F2CF64E037
:105E2000D5CF64E0E5CF68E1DACFCF92DF92EF9291
:105E3000FF920F931F93CF93DF93D62E8C010F5FAA
:105E40001F4F2FE7C22EF8013197E491EE2331F175
:105E5000ED3679F183E0E89FF0011124EF01C85994
:105E6000D74F9BE6E92E98E0F92EEE0EFF1EFE01BD
:105E70006491660FD1106C2581E020DF2196CE154C
:105E8000DF05A9F7DD2099F06FE781E017DF0F5FED
:105E90001F4FF8013197E491EE23D1F6DF91CF91B6
:105EA0001F910F91FF90EF90DF90CF90089560E0E9
:105EB000ECCFDD2089F081E063E400DF81E06BE777
:105EC000FDDE81E067E6FADE81E06BE7F7DE81E088
:105ED00067E4F4DE6FE7D9CF81E06CE3EFDE81E0C9
:105EE00064E0ECDE81E068E1E9DE81E064E0E6DECA
:105EF00081E068E3E3DE60E0C8CFEF92FF920F93AA
:105F00001F93CF93DF93E82EF92EF70101917F01C4
:105F10000023E1F00D3609F183E0089F8001112490
:105F2000E801C859D74F0559174FFE0164916064C5
:105F300081E0C4DE2196C017D107B9F781E060E4A3
:105F4000BDDEF70101917F01002321F7DF91CF91A1
:105F50001F910F91FF90EF90089581E06EE5AEDE06
:105F600081E062E4ABDE81E06CE4A8DE81E062E423
:105F7000A5DE81E06CE5A2DE81E060E49FDEC5CFB6
:105F8000CF93DF93C8EFD1E081E060E097DE219707
:105F9000D9F7DF91CF9108951F9384EB8093E23777
:105FA00084E18093E33784E08093E437569A279A1C
:105FB000259A229A209A2A9880E090E00E94134D18
:105FC000182F815F823018F180E090E062EF0E942C
:105FD0001B4D6091E23781E090E00E941B4D82E012
:105FE00090E060E00E941B4D80E061E267DE60911E
:105FF000E23780E063DE6091E33780E05FDE80E0DF
:1060000060E25CDE80E06CE059DE1F91089581E083
:1060100090E00E94134D8093E237123F29F3D4CFD2
:10602000FC014181842F90E09C01359527952065E6
:106030002CBD40FD06C081E0463019F08DBD2C9886
:10604000089580E08DBD2C980895BF92CF92DF9285
:10605000EF92FF920F931F93CF93DF938C016B010D
:106060007A0120DEEB01BB24BA94BEBC0DB407FE5E
:10607000FDCF8EB5F80182838F3FB1F413DE6C1B28
:106080007D0B81E06D32780780F381E1F801808338
:106090002C9A80E0DF91CF911F910F91FF90EF90AC
:1060A000DF90CF90BF9008958E3F19F08FE08083EE
:1060B000EFCFE114F104F1F00894E108F1088FEF5B
:1060C0008EBDE114F10471F0F60180E090E03FEF45
:1060D0000DB407FEFDCF2EB521933EBD01968E1562
:1060E0009F05B0F30DB407FEFDCF8EB5F601EE0DA2
:1060F000FF1D80838FEF8EBD0DB407FEFDCF8EB5E3
:106100008FEF8EBD0DB407FEFDCF8EB52C9A81E0CA
:10611000C1CF0F931F93CF93DF93EC018B0180DFEF
:10612000CE01B80140E052E090DFDF91CF911F91A6
:106130000F910895FF920F931F93CF93DF93EB017D
:10614000B1DD8B01FF24FA94FEBC0DB407FEFDCF38
:106150008EB58F3F69F0A6DD601B710B6C177D0754
:1061600098F380E0DF91CF911F910F91FF900895F8
:1061700081E0DF91CF911F910F91FF900895DF9201
:10618000EF92FF920F931F93CF93DF93EC01D62EE4
:1061900079018A0145DFCE016CE271E0CBDF8D2D04
:1061A00080648EBD0DB407FEFDCF28E130E0D8013C
:1061B000C701022E04C0B695A795979587950A94B6
:1061C000D2F78EBD0DB407FEFDCF285030408FEFC3
:1061D000283F380761F7DD20E9F08D2D883001F583
:1061E00087E88EBD0DB407FEFDCF8D2D8C30D1F02C
:1061F0002FEF9FEF9EBD0DB407FEFDCF8EB58A83B6
:1062000087FD0AC0DF91CF911F910F91FF90EF9012
:10621000DF90089585E9E5CF2223A1F32150EACF4D
:106220008FEFDFCF8FEF8EBD0DB407FEFDCF8EB5A4
:10623000DFCFCF93DF93EC01F3DECE016CE020E003
:1062400030E0A9019CDF882339F083E088832C9A11
:1062500080E0DF91CF9108952C9A81E0DF91CF917A
:106260000895CF93DF93EC019A01AB018B818330CA
:1062700039F069E0220F331F441F551F6A95D1F78B
:10628000CE0162E17CDF882339F085E088832C9A97
:1062900080E0DF91CF9108952C9A81E0DF91CF913A
:1062A0000895CF92DF92EF92FF920F931F93CF93B7
:1062B000DF93EC017A018B0169018B81833039F026
:1062C000A9E0EE0CFF1C001F111FAA95D1F7CE010B
:1062D00061E1A801970153DF882369F084E0888396
:1062E0002C9A80E0DF91CF911F910F91FF90EF905A
:1062F000DF90CF900895CE01B60140E052E0A5DED8
:10630000F1CF8F929F92BF92CF92DF92EF92FF9246
:106310000F931F93DF93CF930F92CDB7DEB74C014E
:10632000B62EFC0113821082BDDC8B01249A2C9ABC
:106330002698259A279A249A2C9A85E0F40181833D
:1063400082E58CBD1DBC8AE09FEF9EBD0DB407FEAB
:10635000FDCF8150D1F7C40160E020E030E0A90119
:106360000EDF782FF40182838130C9F09BDC601B43
:10637000710BF7E0613D7F0770F381E0F4018083EA
:106380002C9A80E00F90CF91DF911F910F91FF9099
:10639000EF90DF90CF90BF909F908F900895C401B1
:1063A00068E02AEA31E040E050E07983E8DE798174
:1063B00082FF1FC0F4017383CC24DD247601C40165
:1063C00067E320E030E0A901DADEC40169E2A70159
:1063D0009601D5DEF40182838823D9F063DC601B4B
:1063E000710BF7E0613D7F0750F38AE0F401808391
:1063F000C7CF84E02FEF2EBD0DB407FEFDCF9EB5B5
:10640000F40192838150B9F79A3A79F082E080835F
:10641000B7CF83818230B1F02C9AFB2DF73070F02A
:1064200088E1F401808380E0ADCF82E0F4018383D2
:10643000C12CD12CE12CB0E4FB2EC1CFF401B182F0
:1064400081E0A0CFC4016AE320E030E0A90197DE3B
:10645000882321F088E0F401808392CF8FEF8EBDF6
:106460000DB407FEFDCF8EB5807C803C19F483E02F
:10647000F401838383E09FEF9EBD0DB407FEFDCF43
:106480002EB58150C9F7C8CFFC016EBDA42FB52F22
:1064900080E090E00DB407FEFDCF2C912EBD0DB431
:1064A00007FEFDCF11962C9111972EBD02961296E4
:1064B00022E08030920771F70DB407FEFDCF8FEF19
:1064C0008EBD0DB407FEFDCF8FEF8EBD0DB407FE60
:1064D000FDCF8FEF8EBD0DB407FEFDCF8EB582834D
:1064E0008F71853029F083E180832C9A80E00895B4
:1064F00081E008950F931F93CF93DF93EC018B01FD
:106500008FDDCE0168E572E015DE882349F485E170
:1065100088832C9A80E0DF91CF911F910F9108958D
:10652000CE016CEFA801B0DF882389F32C9A81E0BB
:10653000DF91CF911F910F910895CF92DF92EF924B
:10654000FF920F931F93CF93DF93EC017A018B019E
:1065500069018B81833039F089E0EE0CFF1C001F4C
:10656000111F8A95D1F7CE0168E1A801970107DED6
:10657000882369F086E088832C9A80E0DF91CF91B0
:106580001F910F91FF90EF90DF90CF900895CE0173
:106590006EEFA60179DF882379F3CE0168E572E01A
:1065A000C9DD882319F487E18883E6CFCE016DE049
:1065B00020E030E0A901E3DD882319F086E188833B
:1065C000DBCF8FEF8EBD0DB407FEFDCF8EB58823D8
:1065D000A9F72C9A81E0D2CFAF92BF92CF92DF92EF
:1065E000EF92FF920F931F93CF93DF93EC015A0129
:1065F0006B017801890167E320E030E0A901BFDD8C
:10660000CE0167E1A8019701BADD882379F089E01E
:1066100088832C9A80E0DF91CF911F910F91FF909A
:10662000EF90DF90CF90BF90AF9008958B81833033
:1066300039F099E0AA0CBB1CCC1CDD1C9A95D1F753
:10664000CE0169E1A60195019ADD882319F087E062
:106650008883DFCF2C9A81E0DECFCF93DF93EC01EC
:10666000DFDCCE0168E572E065DD882359F08DEF4F
:106670008EBD0DB407FEFDCFCE0168E572E05ADD98
:10668000882339F482E188832C9A80E0DF91CF91CE
:1066900008952C9A81E0DF91CF910895CF93DF93F5
:1066A000EC019C012C5F3F4F898D9A8D41E050E0B9
:1066B00060E070E00E94E03D8823D9F08D899E89DA
:1066C000AF89B88D0097A105B10579F48C819D81C2
:1066D000AE81BF818D8B9E8BAF8BB88F8981806897
:1066E000898381E0DF91CF91089581E0DF91CF919F
:1066F000089580E0DF91CF910895CF92DF92EF92DD
:10670000FF921F93CF93DF93EC0189899A89AB891C
:10671000BC89803E2FEF92072FE1A20720E0B2074D
:1067200048F080E0DF91CF911F91FF90EF90DF90D4
:10673000CF900895CE01B2DF882399F30E94B43B35
:10674000882379F3E98DFA8DCC80DD80EE80FF809F
:106750008EEF9FEFAFEFBFEFC80ED91EEA1EFB1EF4
:10676000058404C0CC0CDD1CEE1CFF1C0A94D2F77F
:1067700086859785A089B189C80ED91EEA1EFB1EA1
:1067800081E08093F139C092EB37D092EC37E09200
:10679000ED37F092EE3780E092E0EFEEF7E3DF01C5
:1067A0009C011D9221503040E1F7E98DFA8D8481E2
:1067B0008230C0F011E006C01F5FE98DFA8D848140
:1067C000181780F4B701A601410F511D611D711DFD
:1067D0008091EF399091F0392FEE37E3AEDE8823C8
:1067E00059F79FCF20E032E040E050E0058404C03C
:1067F000220F331F441F551F0A94D2F789899A89A3
:10680000AB89BC89820F931FA41FB51F898B9A8BFC
:10681000AB8BBC8B81E086CFCF93DF93EC018C8573
:106820009D85AE85BF8541E0662309F440E0BC014B
:10683000CD01DAD7882381F0288930E0220F331F79
:1068400022953295307F3227207F32272151384CD4
:10685000C901DF91CF91089520E030E0C901DF91B7
:10686000CF9108956F927F928F929F92AF92BF9235
:10687000CF92DF92EF92FF920F931F93DF93CF930C
:1068800000D000D0CDB7DEB76C014B013A01DC017E
:106890005596ED90FD900D911C915897E114F104DF
:1068A00001051105F1F05E010894A11CB11C10C096
:1068B000D801C7010196A11DB11D29813A814B81E3
:1068C0005C8182179307A407B507F9F47C018D0159
:1068D000F601818D928DB801A7019501CAD7882351
:1068E00039F780E00F900F900F900F90CF91DF91CC
:1068F0001F910F91FF90EF90DF90CF90BF90AF90DE
:106900009F908F907F906F900895D60159966D91CA
:106910007C915A97FB018789803109F44CC0283F4C
:106920008FEF38078FEF48078FE05807D0F2F60156
:1069300085899689A789B08D0297A109B109FB01C4
:10694000058404C0880F991FAA1FBB1F0A94D2F7A1
:106950002685378540895189820F931FA41FB51F53
:10696000F40180839183A283B383FB01868597859D
:10697000A089B1890197A109B1092481820F911DD4
:10698000A11DB11DA8019701225030404040504048
:10699000058404C0220F331F441F551F0A94D2F7E9
:1069A000820F931FA41FB51FF30180839183A283DD
:1069B000B38381E097CF283FFFEF3F07F0E04F0719
:1069C000F0E05F0708F0B3CF8CCFE82FF92F80E01D
:1069D00090E03EE209C0DB01A90FB11D2C939F5F3F
:1069E0008F5F31968B3061F020812032C9F388307F
:1069F00091F7DB01A90FB11D3C939F5F2081EBCF85
:106A0000690F711DFB01108208951F93FB012BE09C
:106A100030E231932150E9F7A82FB92F30E017E089
:106A20009A2F8B2F2D91222351F4FA019083818389
:106A300081E0FB019081903279F01F9108952F320F
:106A4000A1F32E3261F085EE99E0FC010196E4910C
:106A5000EE2351F02E17C9F780E01F9108951A30E8
:106A6000D9F338E01AE0DCCF1317B0F32132A0F3EA
:106A70002F3790F7FB01E30FF11D822F81568A31EA
:106A800008F4205220833F5FCBCF0F931F93CF9307
:106A9000DF93EC018B018B81882331F4FB01878923
:106AA000803141F08032F1F180E0DF91CF911F9190
:106AB0000F91089582E08B831D8A1E8A1F8A188E8B
:106AC000808D918DA0E0B0E0880F991FAA1FBB1F99
:106AD000880F991FAA1FBB1F880F991FAA1FBB1FD2
:106AE000880F991FAA1FBB1F880F991FAA1FBB1FC2
:106AF000898B9A8BAB8BBC8B1A8F098F81E0898332
:106B00001C821D821E821F82188619861A861B8689
:106B10001C861D861E861F86188ADF91CF911F91C5
:106B20000F91089583E08B83F801428D538D648D1E
:106B3000758D4D8B5E8B6F8B788F9E012F5E3F4FD7
:106B4000C80124D78823C1F6AFCF2F923F924F922E
:106B50005F926F927F928F929F92AF92BF92CF92ED
:106B6000DF92EF92FF920F931F93CF93DF938C01ED
:106B7000362FE72F2A01DC0113962C91139722233D
:106B800029F011968C91119780FD16C02FEF3FEFE1
:106B9000C901DF91CF911F910F91FF90EF90DF908E
:106BA000CF90BF90AF909F908F907F906F905F90AD
:106BB0004F903F902F900895E801C988DA88EB88BC
:106BC000FC88488559856A857B854201AA24BB24B7
:106BD000D701C601841B950BA60BB70B8816990627
:106BE000AA06BB0608F093C04114510409F4BEC0C4
:106BF000832E9E2E6201A4E02A2E312C200E311EFF
:106C0000612CF2E07F2E60C0FF2009F07AC04115B0
:106C100051056105710509F0ABC0E8018D899E89B8
:106C2000AF89B88D8C839D83AE83BF83468557859E
:106C3000608971894F0D511D611D711D0297A10958
:106C4000B109058404C0880F991FAA1FBB1F0A94AD
:106C5000D2F7480F591F6A1F7B1FE301CA19DB09CE
:106C6000CC16DD0608F4E601E2E0C030DE0709F4E8
:106C700052C0CB01BA0140E0B7D5882309F486CFD2
:106C800095012151384CC401B901AE010E94AD4AB1
:106C9000AE0160E070E0F80180859185A285B38542
:106CA000480F591F6A1F7B1FD80118964D935D939B
:106CB0006D937C931B97CC1ADD0A09F457C08C0E98
:106CC0009D1E13962C911397EFEFAE2EE1E0BE2E92
:106CD000A422B5222230B9F1D8015996ED91FC9148
:106CE0005A97DB01CA0129E0B695A7959795879534
:106CF0002A95D1F7F480FA94F822A114B10409F48A
:106D000083CFE8018C819D81AE81BF818FCF260129
:106D1000441A550A69CF8091EB379091EC37A091D6
:106D2000ED37B091EE37481759076A077B0709F42A
:106D3000A0CF8091EF399091F0399401B2DA882395
:106D400009F0A6CF23CF39E07695679557954795FB
:106D50003A95D1F7E801E98DFA8D828D938DA48D56
:106D6000B58D480F591F6A1F7B1F77CF920110CF37
:106D7000D80114964D915D916D917C911797CF013B
:106D8000910177D5882309F401CFE801E98DFA8DC7
:106D90008C819D81AE81BF8149CFDF93CF930F92CC
:106DA000CDB7DEB7BE016F5F7F4F41E050E0CDDE73
:106DB0008130910539F02FEF3FEFC9010F90CF914E
:106DC000DF910895298130E0C9010F90CF91DF91C3
:106DD0000895EF92FF920F931F93CF93DF93EC01EF
:106DE0008B81823050F420E030E0C901DF91CF91F7
:106DF0001F910F91FF90EF900895E884F9840A8520
:106E00001B85CE01CADF97FDEECF88859985AA85BF
:106E1000BB854F96A11DB11D88879987AA87BB871F
:106E2000D801C70115E0B695A795979587951A954E
:106E3000D1F78F70282F30E0220F331F2295329523
:106E4000307F3227207F32272151384CCECF8F928E
:106E50009F92AF92BF92CF92DF92EF92FF920F93E9
:106E60001F93CF93DF93EC014A015B012B81222317
:106E700009F465C089899A89AB89BC89841795070B
:106E8000A607B70708F45BC0223009F452C081148A
:106E90009104A104B10409F46AC0488559856A8542
:106EA0007B85E98DFA8D258530E0275F3F4FDB013B
:106EB000CA010197A109B109022E04C0B695A79590
:106EC000979587950A94D2F7850174010894E10893
:106ED000F1080109110904C016950795F794E79484
:106EE0002A95D2F7E816F9060A071B07B0F58D892F
:106EF0009E89AF89B88D8C839D83AE83BF8384E0E8
:106F0000C82ED12CCC0EDD1E0FC04C815D816E8150
:106F10007F81898D9A8D9601ACD40894E108F1089F
:106F200001091109882359F0E114F1040105110543
:106F300061F788869986AA86BB8681E001C080E0D9
:106F4000DF91CF911F910F91FF90EF90DF90CF9045
:106F5000BF90AF909F908F900895411551056105A6
:106F6000710529F2E81AF90A0A0B1B0BC8CF1C821B
:106F70001D821E821F82188619861A861B8681E052
:106F8000DFCF0F931F93CF93DF93EC018B81882387
:106F900049F0898187FD0EC0E7D3DF91CF911F9122
:106FA0000F91089581E0888380E0DF91CF911F9158
:106FB0000F910895CE0161E02FDC8C01009791F3D1
:106FC000FC018081853E71F38B818230F8F08D89E0
:106FD0009E89AF89B88DF801938F828FB58BA48B72
:106FE000E091E737F091E837309759F0B8016A5EE1
:106FF0007F4FC80148960995F801808D918D938B3C
:10700000828B89818F778983AFD3C7CF89899A890A
:10701000AB89BC89848F958FA68FB78FD8CFCF933C
:10702000DF93EC01AEDF1B82DF91CF9108956F9269
:107030007F928F929F92AF92BF92CF92DF92EF9208
:10704000FF920F931F93DF93CF9300D000D0CDB763
:10705000DEB77C015A016B01DC0113968C9113970A
:107060008130A1F080E00F900F900F900F90CF91A2
:10707000DF911F910F91FF90EF90DF90CF90BF9025
:10708000AF909F908F907F906F90089511968C9104
:10709000119781FFE7CFF70181899289A389B4898C
:1070A00084179507A607B707E8F20097A105B10571
:1070B00029F1F7016084718482849384C701B60149
:1070C000A501C5DE882371F2A114B104C104D10465
:1070D000B9F4D70155964D915D916D917C9158977A
:1070E00059968D919C915A97A3D6882309F4BACFCB
:1070F000F701158A168A178A108E40C081E0B3CF37
:10710000D70114964D915D916D917C911797599689
:107110008D919C915A979E012F5F3F4FAAD3882350
:1071200009F4A0CFD7015996ED91FC915A97498166
:107130005A816B817C8187898031C9F1483F8FEF0B
:1071400058078FEF68078FE07807C0F4CF0170D63B
:10715000882309F487CFD70114964D915D916D91E5
:107160007C91179759968D919C915A970FEF1FEF2D
:107170002FEF3FE086D4882309F474CFF701A18A6A
:10718000B28AC38AD48A818180688183C701F9DE8B
:10719000882309F467CFB601A5016A147B048C0427
:1071A0009D0410F4B401A301C70151DE5CCF483F38
:1071B000BFEF5B07B0E06B07B0E07B07F8F6C6CF28
:1071C0001F93CF93DF93EC01142FE62FF0E0EE0F27
:1071D000FF1FE295F295F07FFE27E07FFE27DF019B
:1071E000A151B84C1B968C911B97817149F0842F4B
:1071F000827131F01B8280E0DF91CF911F91089561
:107200008091EB379091EC37A091ED37B091EE374C
:107210008C879D87AE87BF87688BE151F84C848946
:107220009589A0E0B0E0DC01992788278D8B9E8BA3
:10723000AF8BB88F428D538D60E070E0482B592B97
:107240006A2B7B2B4D8B5E8B6F8B788F838590E0C9
:10725000887190700097F1F4848D958DA68DB78D0F
:10726000898B9A8BAB8BBC8B81E08B83812F8F704A
:1072700089831C821D821E821F82188619861A86A7
:107280001B8614FD17C015FD1EC081E0DF91CF9154
:107290001F9108958031910509F0ACCF9E012F5EBA
:1072A0003F4F898D9A8D72D3882309F4A3CF84E050
:1072B0008B83DCCFCE0140E050E0BA01B8DE8823FA
:1072C00011F780E099CF49895A896B897C89CE0171
:1072D000BEDD92CF8F929F92AF92BF92CF92DF92FC
:1072E000EF92FF920F931F93CF93DF935C01EB011B
:1072F000C42E952E822E898D9A8DD5015A969C93F7
:107300008E935997CB0140E050E0BA01A0DDDD2417
:10731000E884F9840A851B8589899A89AB89BC89A7
:10732000E816F9060A071B0708F040C0CE0151DD38
:10733000FC01009709F476C0D801C70115E0B695A5
:10734000A795979587951A95D1F7182F1F7080816B
:10735000882391F0853E81F08C2D992DBF014BE063
:1073600050E00E94A04A009799F687FC5BC0C501D7
:10737000612F482D25DF57C0DD20A9F42091EB3780
:107380003091EC374091ED375091EE37D5011C9696
:107390002D933D934D935C931F9750961C9350975C
:1073A0008081DD24D394882309F0B2CF86FE3AC0D1
:1073B00081FE38C0DD2009F043C08B81823091F11D
:1073C000CE019BD9882371F1CFEED7E310E07E0187
:1073D000EC2FFF2D80E2DF011D928A95E9F7DE0197
:1073E0008C2D992DFC018BE001900D928150E1F7DD
:1073F000E091E737F091E837309761F1BE01625FC5
:107400007F4FCE0140960995888999892E853F85C1
:107410009B8B8A8B998F888F3F8B2E8BA5D188234E
:1074200009F0A5CF80E0DF91CF911F910F91FF90E0
:10743000EF90DF90CF90BF90AF909F908F90089586
:10744000F5011089C50161E0E7D9EC01009709F069
:10745000BECFE8CF81E298E2998B888B80E098E0FC
:107460009F878E8720E038E081E298E2D1CF2F928B
:107470003F924F925F926F927F928F929F92AF92C4
:10748000BF92CF92DF92EF92FF920F931F93DF9301
:10749000CF93CDB7DEB7C454D0400FB6F894DEBF5B
:1074A0000FBECDBF2C013B018E010E5B1F4FD801DB
:1074B00011965C934E9325962FAF25971C861F86B9
:1074C0001FA21AA66115710509F45FC0FC01838132
:1074D000882309F05AC0CA01DA012C912F3209F42D
:1074E00070C073013CE0832E912C8C0E9D1E6401B4
:1074F0005E010894A11CB11C27E2222E312C2C0E17
:107500003D1EB501A80181DA882369F1D801ED910A
:10751000FC91119780818F3241F43196D8011196F8
:10752000FC93EE9381918F32C9F3882309F46FC0E5
:10753000C601B701A50121E0CDDE8823A1F0E61444
:10754000F70421F0C7011DDDF7011382C814D90427
:10755000C9F076016401D8018D919C91B501A80113
:1075600054DA882399F600E08AA5882321F0CE0119
:10757000879607DD1AA68F85882341F0CE010C96E9
:1075800000DD04C061017401E6CF00E0802FCC5B18
:10759000DF4F0FB6F894DEBF0FBECDBFCF91DF91A6
:1075A0001F910F91FF90EF90DF90CF90BF90AF9021
:1075B0009F908F907F906F905F904F903F902F9013
:1075C00008959A012F5F3F4FC901F801318320834D
:1075D000D9014C912F5F3F4F4F32B1F3F30123811B
:1075E0002250223008F47DCF87E2E82EF12CEC0EF9
:1075F000FD1ED30159966D917C915A97C70145DACA
:10760000882309F4B0CFF801808191816BCFC2014A
:10761000B701A50125962FAD25975CDE082FA4CFD5
:10762000FB01242F6091E5377091E637AF011FCF42
:107630000F931F93CF93DF93EC01662399F08C0196
:107640000E5D1F4F1093E6370093E537C801E7DC66
:10765000BE016C5F7F4FC80118DADF91CF911F9197
:107660000F9108958C010E5D1F4FF0CFDF92EF92C6
:10767000FF920F931F93DF93CF93CDB7DEB76C9735
:107680000FB6F894DEBF0FBECDBFFB01D42E19821A
:107690001C8220812F3229F122E2E22EF12CE80E09
:1076A000F91E8E010F5F1F4FC801B701AF0121E026
:1076B000DEDE8823F1F08C81823070F1D701F80191
:1076C0008BE101900D928150E1F7DD2021F0F092E5
:1076D000E637E092E53721E0C8012C8FA0DC2C8D45
:1076E0000CC021812223C1F6642FA2DF282F8C81B8
:1076F00002C08C8120E0882389F4822F6C960FB61B
:10770000F894DEBF0FBECDBFCF91DF911F910F91D7
:10771000FF90EF90DF90089520E0EDCF8E010F5F96
:107720001F4FDACF0F931F93CF93DF938C010E94EB
:107730008131882331F480E0DF91CF911F910F9147
:107740000895E8012496CE01B80141E0CDD3882305
:1077500021F0C80161E06CDFEFCFCE01B80140E05D
:10776000C3D3882341F3F5CF8091F139882311F4F5
:1077700081E008954091EB375091EC376091ED37FF
:107780007091EE378091EF399091F0392FEE37E319
:107790000E949D32882321F14091F2395091F339B2
:1077A0006091F4397091F539411551056105710504
:1077B00021F41092F13981E008958091EF39909190
:1077C000F0392FEE37E30E949D32882359F0109252
:1077D000F2391092F3391092F4391092F539E9CF59
:1077E00080E0089580E00895DF92EF92FF920F937A
:1077F0001F937B018C01D42E8091EB379091EC3755
:10780000A091ED37B091EE378E159F05A007B10717
:10781000F1F0AADF882339F480E01F910F91FF90E7
:10782000EF90DF9008958091EF399091F039B80191
:10783000A7012FEE37E30E945131882369F3E092CC
:10784000EB37F092EC370093ED371093EE37DD20F5
:1078500049F081E08093F1391F910F91FF90EF90F3
:10786000DF90089581E01F910F91FF90EF90DF90DE
:107870000895CF92DF92EF92FF920F931F93CF93D1
:10788000DF93EC017A018B01690189859A85AB85CB
:10789000BC850196A11DB11D84179507A607B707E2
:1078A00030F0EF89E03169F0E03209F445C080E062
:1078B000DF91CF911F910F91FF90EF90DF90CF90CC
:1078C00008959927872F762F652F2B893C894D891D
:1078D0005E89620F731F841F951F2091EB373091D3
:1078E000EC374091ED375091EE37621773078407FC
:1078F000950729F040E078DF8823C9F2EF89E0316D
:1079000069F18FE790E0A0E0B0E0E822F9220A23D5
:107910001B23F701EE0FFF1FEE0FFF1FE151F84C85
:1079200080819181A281B381BF70F60180839183B0
:10793000A283B38381E0BCCFCB01BA0127E0969547
:107940008795779567952A95D1F72B893C894D893D
:107950005E89620F731F841F951FBFCF8FEF90E06A
:10796000A0E0B0E0E822F9220A231B23F701EE0F82
:10797000FF1FE151F84C80819181A0E0B0E0F60159
:1079800080839183A283B38381E092CF4F925F92F1
:107990006F927F928F929F92AF92BF92CF92DF921F
:1079A000EF92FF920F931F93DF93CF9300D000D0FD
:1079B000CDB7DEB78C0149835A836B837C83290161
:1079C000842F952FA62FB72FAC01BD01CC24DD2429
:1079D00076015E010894A11CB11C612CE2E07E2EB0
:1079E000812C912CC801950144DF882309F447C0FC
:1079F000D401C301F801058404C0880F991FAA1F90
:107A0000BB1F0A94D2F7C80ED91EEA1EFB1E49817D
:107A10005A816B817C818789803119F1483F8FEFD2
:107A200058078FEF68078FE07807E0F2F201C08215
:107A3000D182E282F38281E00F900F900F900F903D
:107A4000CF91DF911F910F91FF90EF90DF90CF903A
:107A5000BF90AF909F908F907F906F905F904F906E
:107A60000895483FFFEF5F07F0E06F07F0E07F0702
:107A7000E8F6C8019501FDDE882309F0B9CF80E062
:107A8000DBCF4F925F926F927F928F929F92AF92D5
:107A9000BF92CF92DF92EF92FF920F931F93CF93FB
:107AA000DF93EC016A017B01280139014230510565
:107AB0006105710590F089859A85AB85BC85019635
:107AC000A11DB11D84179507A607B70730F08F8950
:107AD000803109F456C0803291F080E0DF91CF917F
:107AE0001F910F91FF90EF90DF90CF90BF90AF90DC
:107AF0009F908F907F906F905F904F9008954A0174
:107B00005B0117E0B694A794979487941A95D1F7E0
:107B10008B899C89AD89BE89880E991EAA1EBB1EC1
:107B2000C501B40141E060DE8823B9F28F8980315C
:107B3000A9F18FE790E0A0E0B0E0C822D922EA22C4
:107B4000FB22F601EE0FFF1FEE0FFF1FE151F84C75
:107B500040825182628273828A89823078F18D817B
:107B60009E81AF81B885880D991DAA1DBB1D80938C
:107B7000F2399093F339A093F439B093F53981E059
:107B8000ADCF852E962EA72EBB248B899C89AD89DF
:107B9000BE89880E991EAA1EBB1EC2CF8FEF90E031
:107BA000A0E0B0E0C822D922EA22FB22F601EE0FC3
:107BB000FF1FE151F84C51824082CECF81E08ECF41
:107BC0002F923F924F925F926F927F928F929F92ED
:107BD000AF92BF92CF92DF92EF92FF920F931F93DB
:107BE000DF93CF93CDB7DEB767970FB6F894DEBFBC
:107BF0000FBECDBF1C0149875A876B877C873E87A4
:107C00002D87FC0181859285A385B4859C01AD01FA
:107C10002F5F3F4F4F4F5F4F2D833E834F835887DA
:107C2000ED85FE854080518062807380411451044F
:107C30006104710409F4BEC00894411C511C611C0C
:107C4000711C1F860097A105B10509F454C0D3012A
:107C5000C201CC24DD2476018E010F5F1F4F4C8AB8
:107C60005D8A6E8A7F8A2EC04C015D01C101B5011B
:107C7000A4019801FEDD882309F43DC089819A8121
:107C8000AB81BC810097A105B10509F44EC0A501E7
:107C900094012F5F3F4F4F4F5F4F2C8B3D8B4E8B8F
:107CA0005F8BDA01C9010894C11CD11CE11CF11CD5
:107CB000F1012185328543855485C216D306E40639
:107CC000F506C8F44D805E806F80788448165906AA
:107CD0006A067B0648F682E0882E912CA12CB12CF6
:107CE0008C8A9D8AAE8ABF8AC101B501A401980120
:107CF000C0DD882319F680E067960FB6F894DEBFE2
:107D00000FBECDBFCF91DF911F910F91FF90EF90EC
:107D1000DF90CF90BF90AF909F908F907F906F90AB
:107D20005F904F903F902F900895D501C401019628
:107D3000A11DB11D2C013D012C893D894E895F8912
:107D4000421A530A640A750A29853A854B855C856F
:107D5000421653066406750609F0A5CF4C885D8867
:107D60006E887F88C101B501A4010FEF1FEF2FEFCF
:107D70003FE087DE882309F4BECF481459046A0423
:107D80007B0458F59501840107C0970186014C14C6
:107D90005D046E047F0408F5680179010894C10848
:107DA000D108E108F108C101B701A6016ADE882304
:107DB00061F7A1CFF1014080518062807380F1E0D2
:107DC000FF8729853A854B855C8521303105410542
:107DD000510509F437CF1F8635CFAD85BE854D914E
:107DE0005D916D917C911397411551056105710568
:107DF000C1F4ED85FE854082518262827382FF85E7
:107E0000FF2369F00894411C511C611C711CD101B5
:107E10004D925D926D927C92139781E06DCF81E0DF
:107E20006BCFC101930182012CDE882311F763CF50
:107E3000AF92BF92CF92DF92EF92FF920F931F9378
:107E4000DF93CF9300D000D0CDB7DEB76C017A01BD
:107E50008B0182E090E0A0E0B0E0F60180839183A6
:107E6000A283B3835E010894A11CB11CC601B801B2
:107E7000A7019501FEDC882339F1C601B801A701ED
:107E800000E010E09801FDDD8823F1F0E980FA8040
:107E90000B811C81F6018789803159F088EFE81643
:107EA0008FEFF8068FEF08078FE01807F8F281E0F0
:107EB0000CC0F8EFEF16FFEFFF06F0E00F07F0E061
:107EC0001F07A0F281E001C080E00F900F900F909B
:107ED0000F90CF91DF911F910F91FF90EF90DF9066
:107EE000CF90BF90AF9008956F927F928F929F92A4
:107EF000AF92BF92DF92EF92FF920F931F93CF93B7
:107F0000DF93EC01142F7093F0396093EF391F8ADF
:107F100082E090E0A0E0B0E088839983AA83BB83ED
:107F20001092F1391092F2391092F3391092F4391B
:107F30001092F5398FEF9FEFDC018093EB37909330
:107F4000EC37A093ED37B093EE37442309F444C0E7
:107F5000453078F080E0DF91CF911F910F91FF9035
:107F6000EF90DF90BF90AF909F908F907F906F9039
:107F7000089560E070E0CB0140E036DC882351F3E7
:107F8000212F30E022953295307F3227207F322713
:107F90002152384CF901E254FE4F808190E08F77F6
:107FA00090700097B9F6F901E653FE4F80819181F8
:107FB000A281B38184369105A105B10558F22A53F7
:107FC0003E4FF901E080F18002811381E114F10458
:107FD0000105110521F4BECFEE24FF248701C8015D
:107FE000B70140E001DC882309F4B4CF8091FA376F
:107FF0009091FB37F2E080309F0709F0ABCF2091E2
:10800000FF37222309F4A6CF8091FD379091FE37E8
:10801000009709F49FCF6091FC37662309F49ACF4B
:108020002A8B6C831D8670E080E090E041E050E098
:1080300008C0282F2F5F2D8701968930910509F4FC
:1080400089CFD82E9A01082E02C0220F331F0A941E
:10805000E2F72617370769F76091053870910638FF
:108060006115710509F47FC080E090E06D837E8327
:108070008F8398878090FD379090FE37AA24BB2489
:108080008E0C9F1CA01EB11E8B8A9C8AAD8ABE8A54
:108090006090003870900138798E688E2091FF379B
:1080A00030E040E050E00E94E649680D791D8A1DED
:1080B0009B1D6A8F7B8F8C8F9D8F9301220F331FA7
:1080C00022953295307F3227207F322721503E4F34
:1080D000232F3327269540E050E0260F371F481FF7
:1080E000591F2E873F87488B598B8091023890917A
:1080F0000338009709F440C0A0E0B0E0E21AF30AA8
:10810000040B150BE80EF91E0A1F1B1F04C0169561
:108110000795F794E794DA94D2F7E986FA860B8705
:108120001C8725EFE2162FE0F20620E0020720E090
:10813000120758F185EFE8168FEFF80680E0080780
:1081400080E0180730F180911B3890911C38A09185
:108150001D38B0911E388A8F9B8FAC8FBD8F80E207
:108160008F8B81E0F8CE6091133870911438809134
:108170001538909116387ACF80910F389091103839
:10818000A0911138B0911238B9CF8CE08F8B80E07C
:10819000E2CE80E18F8B81E0DECECF93DF93DC01F6
:1081A000CD91DC9111971C161D06DCF41296E0E0CF
:1081B000F0E020E030E0A901542F432F322F222796
:1081C0006D9170E080E090E0262B372B482B592BE7
:1081D0003196EC17FD0781F7B901CA01DF91CF9104
:1081E000089520E030E0A901F7CFCF93DF93FB01A2
:1081F000DC012D913C91B9016E5F7F4FEC01C60F00
:10820000D71FE60FF71FD9011196A40FB51F21152F
:10821000310599F0215030408A91929141155105D4
:1082200019F06C91862396231197891781F320E02A
:1082300030E0C901DF91CF91089521E030E0C9011C
:10824000DF91CF910895CF93DF93FB01208131819E
:10825000DC012D933C93A081B181109701F1BD0108
:10826000615070401296EA0FFB1FEA01CA0FDB1F34
:10827000A80FB91F80E09A91229130E0290F311D9B
:10828000280F311D81E02F3F310509F008F480E00F
:108290002E93615070409FEF6F3F790761F7DF9138
:1082A000CF910895EF92FF920F931F93CF93DF9397
:1082B0008B01FC01718360836115710581F022E0FF
:1082C000E22EF12CE80EF91EC0E0D0E0C7018C0FC1
:1082D0009D1F0E94AA492196C017D107B9F7DF91C7
:1082E000CF911F910F91FF90EF90089524E030E01F
:1082F000FC013783268384E090E0089521E0FC01AF
:10830000208380E090E00895EF92FF920F931F93F7
:10831000DF93CF930F92CDB7DEB77C018E010F5F55
:108320001F4FC8010E94AA4989818823D1F7F7010C
:108330001782168280E090E00F90CF91DF911F911D
:108340000F91FF90EF9008950F931F93DF93CF93BA
:108350000F92CDB7DEB78C01CE010196FBD7898194
:10836000823070F085E090E0F8019783868325E005
:1083700030E0C9010F90CF91DF911F910F910895C7
:10838000F8019181933141F0882369F481E0F8018B
:10839000828720E030E0EDCF882359F481E08187A7
:1083A00020E030E0E6CF86E0F801828720E030E090
:1083B000E0CF8DE0F801818720E030E0DACF0B9646
:1083C000C9D780E090E00895CF93DF93EC016C89EA
:1083D0007D898E559F4F66DF6C897D89CE018B53D9
:1083E0009F4F60DF80E090E0DF91CF910895FC0126
:1083F0006489758981589F4F55DF80E090E008952A
:108400000F931F93CF93DF938C01EC016696CE01FF
:1084100064E070E047DFCE01C0DEF8016487758755
:108420008687978780E090E0DF91CF911F910F9131
:1084300008950F931F93CF93DF938C01EC01669601
:10844000CE0164E070E02EDFCE01A7DEF801608B84
:10845000718B828B938B695F7F4F8F4F9F4F28E08B
:1084600030E040E050E00E945A4AF801358B248BFE
:108470002132310564F086E090E09783868326E020
:1084800030E0C901DF91CF911F910F91089520E055
:1084900030E0C901DF91CF911F910F910895BC0188
:1084A00081E090E02BD780E090E060E070E026D79C
:1084B00080E090E061E070E021C74F925F926F92A0
:1084C0007F928F929F92AF92BF92CF92DF92EF9264
:1084D000FF920F931F93CF93DF93EC01F62E662349
:1084E00009F4A4C08881861709F4EEC06730C1F092
:1084F0006E30C1F48D30B1F005E010E0C801DF91BD
:10850000CF911F910F91FF90EF90DF90CF90BF9090
:10851000AF909F908F907F906F905F904F90089555
:10852000863051F700E010E0A8E0AA2EFCE0CF2E44
:10853000EEE06E2E7FE0B72E62E0E62E9924939453
:108540005AE0752E45E0D42E37E0832E23E0422EEC
:1085500099E0592EF81691F2873009F495C08830C9
:10856000A8F4833009F453C0843008F03CC0813053
:10857000A1F1823008F454C08F2D893008F49EC0D8
:1085800081E090E08CDF58828881E4CF8B3059F015
:108590008C3078F4893009F467C08A3008F47DC0E3
:1085A0009F2D9B3089F081E090E079DFC88288813F
:1085B000D1CF8D3009F452C08D3000F18E3009F0EA
:1085C00075C09F2D9B30E9F480E090E068DFF88271
:1085D0008881C0CF8F2D813019F181E090E05FDF7D
:1085E000E8828881B7CF853009F444C0863090F0A6
:1085F00081E090E054DF88828881ACCF8F2D8D3070
:1086000019F381E090E04BDFB8828881A3CF9F2DE2
:108610009430D1F281E090E042DFD88288819ACF15
:1086200080E090E03CDF9882888194CF81E090E008
:1086300036DF00E010E080E090E060E070E05ED6C1
:1086400080E090E061E070E059D60F5F1F4F053089
:10865000110589F7188200E010E050CF81E090E02A
:108660001EDF6882888176CF80E090E018DF788214
:10867000888170CF8F2D863009F4A6CF81E090E0FD
:108680000EDFA882888166CF9F2D943009F49CCF9D
:1086900081E090E004DFA882F5CF8F2D813009F4CE
:1086A00093CF81E090E0FBDEE8829BCF8F3009F42E
:1086B00091CFF88205E010E088814CCF80E090E017
:1086C000EEDE4882888146CF863049F08D3009F051
:1086D00029CF81E090E0E3DE8EE0888323CF81E044
:1086E00090E0DDDE87E088831DCFCF92DF92EF92AE
:1086F000FF920F931F93CF93DF93EC018C010A5EDF
:108700001F4FC80161E070E0CDDDC88CC80161E099
:1087100070E0C8DDD88CC80164E070E0C3DDC8013A
:108720003CDD7B018C0188858C1521F0CE010896FB
:108730006C2DC3DEC801B70123D688858D1521F0C5
:10874000CE0108966D2DB9DE80E090E0DF91CF91EB
:108750001F910F91FF90EF90DF90CF9008950F93AE
:108760001F93DF93CF930F92CDB7DEB78C01CE016D
:108770000196F0D5C801089669819FDE9C0100979B
:1087800019F0F80197838683C9010F90CF91DF918B
:108790001F910F9108954F925F926F927F928F92E7
:1087A0009F92AF92BF92CF92DF92EF92FF920F9380
:1087B0001F93CF93DF935B016C01FA013801211500
:1087C000310509F481C080819181D90111969C9372
:1087D0008E93808191818C010E5F1F4F020F131FBA
:1087E000A114B104C104D10409F45DC022E0422EF9
:1087F000512C480E591E4E0E5F1E0CC0011511055E
:1088000019F0D8019E928D01A114B104C104D104C4
:1088100009F449C0F20182902F01EE24FF2499242B
:108820000894A108B108C108D1086114710429F0A5
:10883000A114B104C104D10481F1C82DD0E0BE015E
:108840006170707082E090E059D580E090E060E067
:1088500070E054D50115110549F08ED590E00E2C2D
:1088600002C0880F991F0A94E2F7982A80E090E0EE
:1088700061E070E043D5A114B104C104D10409F44E
:10888000BDCF0894E11CF11CF8E0EF16F10409F4E7
:10889000B5CFD595C7958C2EC3CF81E090E061E030
:1088A00070E02CD5CACFDF91CF911F910F91FF902F
:1088B000EF90DF90CF90BF90AF909F908F907F9080
:1088C0006F905F904F9008958081918100E010E05B
:1088D00087CF2F923F924F925F926F927F928F92AB
:1088E0009F92AF92BF92CF92DF92EF92FF920F933F
:1088F0001F93DF93CF93CDB7DEB728970FB6F894C9
:10890000DEBF0FBECDBF3C01962E29833A834B8339
:108910005C831E830D8317012601B886AF82A9A050
:1089200051E0C52ED12C681509F487C029813A8100
:108930004B815C81211531054105510529F58D8D4E
:108940009E8DAF8DB8A10097A105B10509F097C024
:1089500020E030E0C90128960FB6F894DEBF0FBEC4
:10896000CDBFCF91DF911F910F91FF90EF90DF90DE
:10897000CF90BF90AF909F908F907F906F905F90BF
:108980004F903F902F900895BB24EE24FF24C30105
:10899000692D93DD69817A818B819C814D815E8116
:1089A00091018601F8DE4114510461F0C201B10168
:1089B0004F8158851ADC41E0E42EF12C009711F02C
:1089C000EE24FF24C114D104E9F0D3018C918F5F10
:1089D0008C93E114F10459F02D8D3E8D4F8D58A1EB
:1089E000211531054105510511F0BA1448F1C301B3
:1089F000682D63DD8D8D9E8DAF8DB8A10097A1058B
:108A0000B10591F4E114F10409F4A2CFB3948B2DD4
:108A100081508A1508F4BBCFAA2019F0AB1408F4D2
:108A200039C022E030E096CFC30161E046DD6D8DB4
:108A30007E8D8F8D98A1A4D4E5CFCC24DD2476CF74
:108A4000C30166E03ADDC30164E037DD8D8D9E8DA4
:108A5000AF8DB8A1B595A79597958795B595A7952D
:108A6000979587952D8D3E8D4F8D58A1280F391FD5
:108A70004A1F5B1F2D8F3E8F4F8F58A3BBCFC30163
:108A800061E01BDD6D8D7E8D8F8D98A179D420E006
:108A900030E060CF23E030E05DCF8F92AF92BF92A5
:108AA000CF92DF92EF92FF920F931F93CF93DF93BA
:108AB000EC018C010A5E1F4F6C897D89C801F2DBD5
:108AC00000D000D00F92288939894A895B89ECE56A
:108AD000EE2EF12CEC0EFD1E79E3C72ED12CCC0E20
:108AE000DD1E6FE7A62EB12CAC0EBD1E8C859D85BC
:108AF000AE85BF85EDB7FEB781839283A383B48330
:108B00008B858583CE01089664E08A84E2DE9C0131
:108B10000F900F900F900F900F90009711F09F8380
:108B20008E83C901DF91CF911F910F91FF90EF903C
:108B3000DF90CF90BF90AF908F9008958F92AF92BB
:108B4000BF92CF92DF92EF92FF920F931F93CF933A
:108B5000DF93EC018C010A5E1F4FC80162E070E0F8
:108B6000A1DBC8011ADB6B017C01695F7F4F8F4F6E
:108B70009F4F28E030E040E050E09CD421323105A6
:108B80008CF026E030E03F832E83C901DF91CF9146
:108B90001F910F91FF90EF90DF90CF90BF90AF901B
:108BA0008F900895C801B9017DDB00D000D00F92ED
:108BB0008C859D85AE85BF85EDB7FEB78183928399
:108BC000A383B4831582CE0108966BE0A7019601BA
:108BD000EE24FF24CC24DD24AA24BB24898479DE5E
:108BE0009C010F900F900F900F900F90009769F2DB
:108BF000CACF6F927F928F92AF92BF92CF92DF9245
:108C0000EF92FF920F931F93DF93CF930F92CDB705
:108C1000DEB73C01CE0101969DD383010A5E1F4F52
:108C2000298130E040E050E0295F3F4F4F4F5F4FD8
:108C3000F3E05595479537952795FA95D1F7C801F3
:108C4000B90130DB00D000D00F92298130E040E044
:108C500050E0F30184859585A685B785EDB7FEB70D
:108C600081839283A383B4831582C30108966BE04A
:108C7000EE24FF24CC24DD24AA24BB24F301818428
:108C800028DE9C010F900F900F900F900F9000978F
:108C900019F0F30197838683C9010F90CF91DF917B
:108CA0001F910F91FF90EF90DF90CF90BF90AF900A
:108CB0008F907F906F9008952F923F924F925F9286
:108CC0006F927F928F92AF92BF92CF92DF92EF928C
:108CD000FF920F931F93DF93CF9300D0CDB7DEB7F2
:108CE0009A8389831A012B013901C801B901DADAA3
:108CF000C114D10419F0C601B301D4DA00D000D0F8
:108D00000F928E899F89A88DB98DEDB7FEB78183AB
:108D10009283A383B4838A8D858389819A8164E059
:108D2000A2019101D6DD0F900F900F900F900F9040
:108D30000F900F90CF91DF911F910F91FF90EF90C7
:108D4000DF90CF90BF90AF908F907F906F905F90AB
:108D50004F903F902F9008958F92AF92BF92CF92F5
:108D6000DF92EF92FF920F931F93CF93DF93EC016B
:108D700089818131D9F114E0812E00D000D00F9289
:108D8000488959896A897B892C893D898E010A5EC7
:108D90001F4FBCE5EB2EF12CEC0EFD1EA9E3CA2EF5
:108DA000D12CCC0EDD1EEDB7FEB7118212821382DC
:108DB00014821582CE010896AA24BB247DDF9C0173
:108DC0000F900F900F900F900F90009711F09F83CE
:108DD0008E83C901DF91CF911F910F91FF90EF908A
:108DE000DF90CF90BF90AF908F9008958A84C5CFC9
:108DF0008F92AF92BF92CF92DF92EF92FF920F933A
:108E00001F93CF93DF93EC0189818E30A9F104E0A9
:108E1000802E00D000D00F92488959896A897B89B9
:108E20002C893D898E010A5E1F4FEDB7FEB7118276
:108E30001282138214821582CE010896EE24FF243A
:108E4000CC24DD24AA24BB2437DF9C010F900F9093
:108E50000F900F900F90009711F09F838E83C901A0
:108E6000DF91CF911F910F91FF90EF90DF90CF9006
:108E7000BF90AF908F9008958A84CBCF8F92AF929E
:108E8000BF92CF92DF92EF92FF920F931F93CF93F7
:108E9000DF93EC0100D000D00F92488959896A898C
:108EA0007B892C893D898C010A5E1F4FECE5EE2EF3
:108EB000F12CE80EF91E99E3C92ED12CCC0EDD1E43
:108EC0008FE7A82EB12CAC0EBD1E8C859D85AE857E
:108ED000BF85EDB7FEB781839283A383B4838B856F
:108EE0008583CE0108968A84E7DE9C010F900F905F
:108EF0000F900F900F90009711F09F838E83C90100
:108F0000DF91CF911F910F91FF90EF90DF90CF9065
:108F1000BF90AF908F900895CF92DF92EF92FF9223
:108F20000F931F93CF93DF938C016B017901B801ED
:108F30008AD9E60128813981F701A081B181AD018B
:108F40004150504057FD38C0FD013296EE0DFF1DD7
:108F50001196A00FB11F60E010E08291882329F1E3
:108F6000EC9001E00AC0762F660F7123B1F0E02A81
:108F7000959587958823C1F0000F90E080FFF8CF8A
:108F8000662389F721503040B601620F731FEB0151
:108F90001A8162E071E0712351F7702F7095E7221A
:108FA00095958795882341F7EC9241505040119751
:108FB0008FEF4F3F580789F6DF91CF911F910F91A7
:108FC000FF90EF90DF90CF9008952F923F924F92B5
:108FD0005F926F927F928F929F92AF92BF92CF9249
:108FE000DF92EF92FF920F931F93DF93CF93CDB752
:108FF000DEB761970FB6F894DEBF0FBECDBF3C0160
:10900000B6E14B2E512C480E591EFC01648975891E
:10901000C20148D9C30108969D838C83F301E45AA9
:10902000FF4FFF83EE83C301C99699878887AFE717
:109030002A2E312C260C371C00D000D00F92F301C1
:10904000208931894289538984859585A685B7858C
:10905000EDB7FEB781839283A383B483F301838545
:10906000EDB7FEB785838C819D8164E08201EE803F
:10907000FF80C884D9845101F30182842ADC9B8358
:109080008A830F900F900F900F900F90009709F028
:1090900087C0C3018B539F4F9D878C87FC01408104
:1090A0005181141615060CF09DC0E0E0F0E060E080
:1090B00000E010E0E60DF71DE953FF4F80818823A3
:1090C00051F090E09C0121703070020F131F9595B4
:1090D00087958823B1F76F5FE62FF0E0E417F50777
:1090E0004CF3CE01019636D1222717FD2095322F61
:1090F000095F1F4F2F4F3F4FE3E035952795179599
:109100000795EA95D1F71F870E879924C3018851E7
:109110009F4F9B878A87F301EE55FF4FF98BE88BB2
:109120008981981608F043C08A859B856E857F8566
:10913000B9D8C2016A857B85488959892C853D85C6
:10914000EBDE00D000D00F92F301208931894289F3
:10915000538984859585A685B785EDB7FEB781834C
:109160009283A383B483F3018385EDB7FEB7858330
:109170008C819D8164E08201EE80FF80C884D98467
:109180005101F3018284A5DB0F900F900F900F9097
:109190000F90009739F493948981981640F4C4CFC6
:1091A0008A819B81F301978386839B838A838A814B
:1091B0009B8161960FB6F894DEBF0FBECDBFCF91F5
:1091C000DF911F910F91FF90EF90DF90CF90BF90B4
:1091D000AF909F908F907F906F905F904F903F9057
:1091E0002F90089500E010E07CCFCF93DF93EC0147
:1091F000188219821A821B821C821D821F821E8283
:109200001B86188681E089878A87188A198A1A8AB4
:109210001B8A1D8A1C8A1C861D861E861F86CE01FF
:10922000089660E04AD98E839F83DF91CF9108959D
:10923000CF93DF93EC012E813F812115310519F485
:109240008881882321F0C901DF91CF910895CE0153
:10925000019680D08A819B81AC81BD810196A11D40
:10926000B11D8A839B83AC83BD83E981E83150F0D3
:1092700084E090E09F838E8324E030E0C901DF9199
:10928000CF910895F0E0EE0FFF1FED51FB4F0190DD
:10929000F081E02DCE0109952E813F81D4CF0F932F
:1092A0001F93DF93CF93CDB7DEB7CB50D1400FB62E
:1092B000F894DEBF0FBECDBF8E010F5F1F4FC801F8
:1092C00094DF2F8138852115310569F0C901C55F0B
:1092D000DE4F0FB6F894DEBF0FBECDBFCF91DF914A
:1092E0001F910F9108958981882381F7C801A0DF1C
:1092F0002F81388521153105B1F3E8CF81309105F3
:1093000051F08230910561F0009721F461157105EB
:1093100071F4429808956115710539F0439A0895E2
:109320006115710531F0459A089543980895429A60
:1093300008954598089580E090E060E070E0DEDFF9
:1093400080E090E061E070E0D9CF9093F7398093AE
:10935000F6390895CF93DF93EC01E091F639F0915F
:10936000F739309729F009958883DF91CF910895D7
:109370001882DF91CF91089581E0349B80E00895B9
:10938000AF92BF92CF92DF92EF92FF920F931F9313
:109390005B016C01161617061806190674F4EE2404
:1093A000FF248701C8DF0894E11CF11C011D111D79
:1093B000EA14FB040C051D05ACF31F910F91FF90FF
:1093C000EF90DF90CF90BF90AF900895629FD00153
:1093D000739FF001829FE00DF11D649FE00DF11D70
:1093E000929FF00D839FF00D749FF00D659FF00D1F
:1093F0009927729FB00DE11DF91F639FB00DE11D0C
:10940000F91FBD01CF0111240895991B79E004C013
:10941000991F961708F0961B881F7A95C9F78095B3
:109420000895AA1BBB1B51E107C0AA1FBB1FA617AB
:10943000B70710F0A61BB70B881F991F5A95A9F7FD
:1094400080959095BC01CD01089597FB092E0726C4
:109450000AD077FD04D0E5DF06D000201AF470951D
:1094600061957F4F0895F6F7909581959F4F0895E8
:10947000A1E21A2EAA1BBB1BFD010DC0AA1FBB1F18
:10948000EE1FFF1FA217B307E407F50720F0A21B8A
:10949000B30BE40BF50B661F771F881F991F1A94F7
:1094A00069F760957095809590959B01AC01BD0121
:1094B000CF01089597FB092E05260ED057FD04D045
:1094C000D7DF0AD0001C38F450954095309521958F
:1094D0003F4F4F4F5F4F0895F6F7909580957095E9
:1094E00061957F4F8F4F9F4F08950790F691E02D24
:1094F00009949111089581568A5108F48052855833
:109500000895FB01DC0105900D920020E1F708951C
:10951000FC0105900020E9F7809590958E0F9F1F24
:109520000895FB01DC014150504048F005900D9238
:109530000020C9F701C01D9241505040E0F7089546
:10954000FB01DC0104C08D910190801921F4415090
:109550005040C8F7881B990B0895FB01DC0102C03D
:1095600001900D9241505040D8F70895FB01DC0165
:109570004150504030F08D910190801919F4002035
:10958000B9F7881B990B0895FB01DC01415050404D
:1095900048F001900D920020C9F701C01D92415082
:1095A0005040E0F708950F931F93DF93CF93CDB70B
:1095B000DEB72E970FB6F894DEBF0FBECDBF0D8974
:1095C0001E898F89988D26E02C831A83098397FF43
:1095D00002C080E090E801979E838D839E01255E06
:1095E0003F4FCE010196698D7A8DA90119D04D8129
:1095F0005E8157FD0AC02F813885421753070CF44E
:109600009A01020F131FF80110822E960FB6F894DC
:10961000DEBF0FBECDBFCF91DF911F910F91089597
:109620002F923F924F925F926F927F928F929F9272
:10963000AF92BF92CF92DF92EF92FF920F931F9360
:10964000DF93CF93CDB7DEB72C970FB6F894DEBF7C
:109650000FBECDBF6C011B018A01FC01178216826F
:10966000838181FFC4C12E010894411C511CF60165
:109670009381F10193FD859193FF81911F018823CF
:1096800009F4B1C1853239F493FD859193FF81913D
:109690001F01853221F490E0B601F5D1E8CFEE2428
:1096A000FF2420E02032B0F48B3269F08C3228F4B1
:1096B000803251F0833271F40BC08D3239F0803337
:1096C00049F421602CC02260246029C0286027C092
:1096D000206125C027FD2CC0382F30533A3098F434
:1096E00026FF08C08E2D880FE82EEE0CEE0CE80E3B
:1096F000E30E15C08F2D880FF82EFF0CFF0CF80E0F
:10970000F30E20620CC08E3221F426FD6CC1206461
:1097100006C08C3611F4206802C0883649F4F10185
:1097200093FD859193FF81911F01882309F0BACFA2
:10973000982F9554933018F09052933028F40C5F82
:109740001F4FFFE3F9830DC0833631F0833771F08B
:10975000833509F05CC021C0F801808189830E5FE8
:109760001F4F420171E0A72EB12C15C062E0662E9A
:10977000712C600E711EF8018080918026FF03C05D
:109780006E2D70E002C06FEF7FEFC4012C8770D1A7
:109790005C0183012C852F7716C052E0652E712C59
:1097A000600E711EF8018080918026FF03C06E2D2F
:1097B00070E002C06FEF7FEFC4012C874ED15C01D7
:1097C0002C852068830123FD1EC007C080E290E045
:1097D000B6012C8758D1FA942C858F2D90E0A816CD
:1097E000B906A0F310C0F40127FD859127FF8191F0
:1097F0004F0190E0B6012C8746D12C85F110FA94E8
:109800000894A108B108A114B10469F7E9C084362D
:1098100011F0893641F527FF08C0F8016081718198
:10982000828193810C5F1F4F09C0F80160817181B3
:10983000882777FD8095982F0E5F1F4F4FE6B42E37
:10984000B22297FF09C090958095709561957F4FE2
:109850008F4F9F4FF0E8BF2AA2012AE030E03FD1AE
:10986000782E741844C0853731F43FEEB32EB222FF
:109870002AE030E025C099EFB92EB2228F36C1F030
:10988000803720F4883509F0AEC00DC0803721F054
:10989000883709F0A8C002C020E1B22AB4FE0BC08C
:1098A00084E0B82A08C0B4FE09C0E6E0BE2A06C0BB
:1098B00028E030E005C020E130E002C020E132E0E5
:1098C000B7FE08C0F80160817181828193810C5FCD
:1098D0001F4F07C0F8016081718180E090E00E5F4A
:1098E0001F4FA201FCD0782E7418FFE7BF22B6FEEE
:1098F0000BC02EEFB2227E1438F4B4FE07C0B2FCC7
:1099000005C08FEEB82202C0A72C01C0AE2C8B2D53
:1099100090E0B4FE0DC0FE01E70DF11D2081203363
:1099200019F4E9EEBE2209C0A394B2FE06C004C039
:1099300086789070009709F0A3948B2C9924B3FC3F
:1099400013C0B0FE0EC0AF1428F4E72CEF0CEA18D9
:10995000AF2C07C0E72C05C080E290E0B60193D0A1
:10996000A394AF14C8F304C0AF1410F4FA1801C0E4
:10997000FF2484FE0EC080E390E0B60184D082FE16
:109980001DC081FE03C088E590E010C088E790E02C
:109990000DC0C40186789070009781F081FC02C0F0
:1099A00080E201C08BE2B7FC8DE290E0B6016BD0A3
:1099B00005C080E390E0B60166D0EA947E14C8F357
:1099C0007A94F201E70DF11D808190E0B6015BD041
:1099D0007720B1F705C080E290E0B60154D0FA9448
:1099E000FF20C9F744CEF6012681378102C02FEF50
:1099F0003FEFC9012C960FB6F894DEBF0FBECDBF66
:109A0000CF91DF911F910F91FF90EF90DF90CF905A
:109A1000BF90AF909F908F907F906F905F904F908E
:109A20003F902F900895F999FECF92BD81BDF89A8D
:109A3000992780B50895262FF999FECF92BD81BD53
:109A4000F89A019700B4021639F01FBA20BD0FB67C
:109A5000F894FA9AF99A0FBE0895FC0105906150A6
:109A600070400110D8F7809590958E0F9F1F089534
:109A7000FC016150704001900110D8F780959095DD
:109A80008E0F9F1F08950F931F93CF93DF938C0129
:109A9000EB018B8181FF1BC082FF0DC02E813F81B6
:109AA0008C819D812817390764F4E881F98101933D
:109AB000F983E88306C0E885F985802F099500972A
:109AC00031F48E819F8101969F838E8302C00FEFB8
:109AD0001FEFC801DF91CF911F910F910895FA01F7
:109AE000AA27283051F1203181F1E8946F936E7FDD
:109AF0006E5F7F4F8F4F9F4FAF4FB1E03ED0B4E0CE
:109B00003CD0670F781F891F9A1FA11D680F791F0E
:109B10008A1F911DA11D6A0F711D811D911DA11D1F
:109B200020D009F468943F912AE0269F112430192F
:109B3000305D3193DEF6CF010895462F4770405DCA
:109B40004193B3E00FD0C9F7F6CF462F4F70405D79
:109B50004A3318F0495D31FD4052419302D0A9F7D4
:109B6000EACFB4E0A6959795879577956795BA95CE
:109B7000C9F700976105710508959B01AC010A2E94
:109B800006945795479537952795BA95C9F7620F6B
:109B9000731F841F951FA01D089519E000E0C8EFF2
:109BA000D9E040E005C022974109FE014BBF9DDC92
:0C9BB000CA3FD1074007B9F7F894FFCF77
:109BBC0025750053442072656164206572726F7262
:109BCC002052004241442046555345532025303203
:109BDC0058202530325820253032580043504C4400
:109BEC0020495320424C414E4B0057524F4E472078
:109BFC0043504C44202D2025640053454C462D5495
:109C0C00455354204F4B006669726D776172652E17
:109C1C0078766600524553554C543A20535543437D
:109C2C00455353004649524D5741524520455252D7
:109C3C004F522025640043504C44204669726D7786
:109C4C006172652025640025640053656C6563743E
:109C5C002044656661756C74204D6F6465004E4FD1
:109C6C0020534420434152443F0043415244204539
:109C7C0052524F522025643A2564002564202564F5
:109C8C0020256420256420256420256400696E63EA
:109C9C006F6D706C657465207772697465006261B4
:109CAC006420736563746F7220256420666F722064
:109CBC0074256400627566206C6F636B6564202587
:109CCC00642F25643A256400636865636B73756D56
:109CDC00206661696C757265203000636865636B22
:109CEC0073756D206661696C7572652031006368EF
:109CFC0065636B73756D206661696C757265203276
:109D0C0000636865636B73756D206661696C0053E5
:109D1C004420726561642073746172742065727280
:109D2C006F720053442072656164206572726F72A9
:109D3C0020440077722077726F6E672074726163B3
:109D4C006B2025642F2564005265766572746564FA
:109D5C002074726B20253032642020200053442064
:109D6C0072656164206572726F72205700534420D3
:109D7C0077726974655374617274206661696C00E2
:109D8C005344207772697465206572726F72005348
:109D9C004420777269746553746F70206661696CC6
:109DAC000053617665642074726B20253032642018
:109DBC00696E20256C7520200025303264002564E6
:109DCC00200053442072656164206572726F7220AA
:109DDC005200D5AAAD0000000000000000000000F9
:109DEC00008A01AD01D8010D024E023078393620BF
:109DFC0053594E4300444154412053495A453F0066
:109E0C00524553504F4E53452053495A453F004FEE
:109E1C0056455252554E00524541442053544154DC
:109E2C0045204348414E47454420256400454E4358
:109E3C004F44452053495A4500524553504F4E53B9
:109E4C00452053495A45203100524553504F4E53EB
:109E5C00452053495A45203200524553504F4E53DA
:109E6C004520544F4F2042494700554E4B20434FFD
:109E7C004D4D414E44004E4F2044415441004752F9
:109E8C004F5550212025303258202530325820256E
:109E9C003032580025303258200049474E4F524539
:109EAC00442025642C20574320256400253032584B
:109EBC0000434D4420434845434B53554D00636D7F
:109ECC006420253032583A20253032582025303243
:109EDC005800484432302E64736B0043616E277413
:109EEC002066696E6420257300256C75204D420038
:109EFC0048442053442072656164206572726F720D
:109F0C00004844205344207772697465537461721D
:109F1C0074206661696C0048442053442077726950
:109F2C007465206572726F72004844205344207728
:109F3C007269746553746F70206661696C00525558
:109F4C004E542057524954450042414420434D44FD
:109F5C0020535A3F2025642025303258202530329A
:109F6C0058002E2E0053656C656374204469736B26
:109F7C00006E6F20696D6167652066696C65732082
:109F8C00666F756E640001030507090E1012141636
:109F9C00181C1E7E41F741F9454D4500427641762D
:109FAC0041DF4119423E47E441E547F846F846F89F
:109FBC0046AC46AC46AC46AF43A441A4419E458456
:049FCC004175430098
:020000021000EC
:08EFF800DDDDDDDD000100009C
:00000001FF
